:020000040000FA
:060000003AEF4CF0120083
:020006001200E6
:06000800D9EF47F01200E1
:02000E000200EE
:10001000EE980000C400000017000000EC980000FB
:080020005E0000000200000078
:08002800D9CFE6FFE1CFD9FFBB
:1000300081E946E800010051680A02E102EF1BF085
:100040000F0A02E12BEF1AF0010A02E154EF19F056
:10005000030A02E17DEF18F0010A02E1D8EF16F081
:10006000530A02E17CEF16F0010A02E120EF16F0DC
:10007000030A02E1C4EF15F0010A02E157EF15F09F
:10008000070A02E1F7EF14F0010A02E197EF14F01A
:10009000030A02E13FEF14F0010A02E1E7EF13F077
:1000A0001F0A02E18FEF13F0010A02E133EF13F0B0
:1000B000030A02E1D7EF12F0010A02E17BEF12F02E
:1000C000070A02E11FEF12F0010A02E1BFEF11F08F
:1000D000030A02E173EF11F0010A02E1A7EF0EF04B
:1000E000700A02E127EF0EF00F0A02E1D1EF0DF0E6
:1000F000010A02E17BEF0DF0030A02E125EF0DF0AA
:10010000010A02E1BBEF0CF0070A02E155EF0CF027
:10011000010A02E1FBEF0BF0030A02E196EF0BF09C
:10012000010A02E1EAEF09F0470A02E187EF09F06C
:10013000010A02E107EF09F0030A02E18AEF08F081
:10014000010A02E1CAEF06F01B0A02E16BEF06F0BA
:10015000010A02E110EF06F0030A02E1B5EF05F033
:10016000010A02E15AEF05F0070A02E1FFEF04F08D
:10017000010A01E1E9D30E0A01E18BD3070A01E18B
:100180002DD3010A01E120D2030A01E136D1010A8F
:1001900002E0D9EF1BF0000101513AE00001060531
:1001A0000DE1AB0EE66E730EE66EE66A600EE66E6D
:1001B000000EE66E80EC49F045E920D0020E000109
:1001C000065D0DE1960EE66E730EE66EE66A600E53
:1001D000E66E000EE66E80EC49F045E90FD00001B6
:1001E00006510CE1810EE66E730EE66EE66A600E55
:1001F000E66E000EE66E80EC49F045E9E66A600EB8
:10020000E66E000EE66E90EC1CF043E900C001F0D3
:10021000000106052BE108C0E6FF09C0E6FFD95042
:10022000010FE66EDACFE6FF05EC1DF044E9C40EDF
:10023000E66E000EE66ED950010FE66EDACFE6FFED
:100240006E0EE66E730EE66EE66A600EE66E000EE9
:10025000E66E80EC49F049E9400EE66E600EE66E0F
:10026000000EE66E90EC1CF043E909D0400EE66EFD
:10027000C60EE66E000EE66E90EC1CF043E9700EC2
:1002800000011F1902E1170E201911E1C40EE66EDC
:10029000000EE66E580EE66E730EE66EE66A600EAF
:1002A000E66E000EE66E80EC49F047E93DD0880E20
:1002B00000011F1902E1130E201911E1C40EE66EB0
:1002C000000EE66E420EE66E730EE66EE66A600E95
:1002D000E66E000EE66E80EC49F047E925D021C0BD
:1002E000E6FF22C0E6FFD950010FE66EDACFE6FF47
:1002F00005EC1DF044E9C40EE66E000EE66ED95022
:10030000010FE66EDACFE6FFC40EE66E000EE66E73
:100310002E0EE66E730EE66EE66A600EE66E000E58
:10032000E66E80EC49F04BE9140EE66E600EE66E68
:10033000000EE66E90EC1CF043E9700E00013119DE
:1003400002E1170E321911E1C40EE66E000EE66EE0
:10035000180EE66E730EE66EE66A600EE66E000E2E
:10036000E66E80EC49F047E93DD0880E0001311976
:1003700002E1130E321911E1C40EE66E000EE66EB4
:10038000020EE66E730EE66EE66A600EE66E000E14
:10039000E66E80EC49F047E925D033C0E6FF34C073
:1003A000E6FFD950010FE66EDACFE6FF05EC1DF04F
:1003B00044E9C40EE66E000EE66ED950010FE66EFB
:1003C000DACFE6FFC40EE66E000EE66EEE0EE66EC7
:1003D000720EE66EE66A600EE66E000EE66E80EC69
:1003E00049F04BE9540EE66E600EE66E000EE66EC6
:1003F00090EC1CF043E9DAEF1BF00001010516E078
:10040000D90EE66E720EE66EE66A600EE66E000EBD
:10041000E66E80EC49F045E9E66A600EE66E000E95
:10042000E66E90EC1CF043E900C001F000010651BB
:100430000DE1C40EE66E720EE66EE66A600EE66EC2
:10044000000EE66E80EC49F045E931D000013C51E8
:100450000DE1AF0EE66E720EE66EE66A600EE66EB7
:10046000000EE66E80EC49F045E921D03AC0E6FF87
:100470003BC0E6FFD950010FE66EDACFE6FF05EC90
:100480001DF044E9C40EE66E000EE66ED950010F71
:10049000E66EDACFE6FF9C0EE66E720EE66EE66A58
:1004A000600EE66E000EE66E80EC49F049E9400E03
:1004B000E66E600EE66E000EE66E90EC1CF043E910
:1004C000700E00012B1902E1170E2C1911E1C40E58
:1004D000E66E000EE66E860EE66E720EE66EE66A5A
:1004E000600EE66E000EE66E80EC49F047E93DD006
:1004F000880E00012B1902E1130E2C1911E1C40E14
:10050000E66E000EE66E700EE66E720EE66EE66A3F
:10051000600EE66E000EE66E80EC49F047E925D0ED
:100520002DC0E6FF2EC0E6FFD950010FE66EDACFF0
:10053000E6FF05EC1DF044E9C40EE66E000EE66E23
:10054000D950010FE66EDACFE6FFC40EE66E000E5C
:10055000E66E5C0EE66E720EE66EE66A600EE66EA3
:10056000000EE66E80EC49F04BE9140EE66E600E6C
:10057000E66E000EE66E90EC1CF043E98BA40DD005
:10058000470EE66E720EE66EE66A600EE66E000ECE
:10059000E66E80EC49F045E90CD0320EE66E720E44
:1005A000E66EE66A600EE66E000EE66E80EC49F0DE
:1005B00045E9540EE66E600EE66E000EE66E90ECB7
:1005C0001CF043E9DAEF1BF0020E0001015D16E0BA
:1005D0001D0EE66E720EE66EE66A600EE66E000EA8
:1005E000E66E80EC49F045E9E66A600EE66E000EC4
:1005F000E66E90EC1CF043E900C001F0030E000130
:100600003C5D0DE1080EE66E720EE66EE66A600E67
:10061000E66E000EE66E80EC49F045E955D0700EAE
:100620000001251902E1170E261911E1C40EE66E2C
:10063000000EE66EF20EE66E710EE66EE66A600E73
:10064000E66E000EE66E80EC49F047E93DD0880E7C
:100650000001251902E1130E261911E1C40EE66E00
:10066000000EE66EDC0EE66E710EE66EE66A600E59
:10067000E66E000EE66E80EC49F047E925D027C013
:10068000E6FF28C0E6FFD950010FE66EDACFE6FF9D
:1006900005EC1DF044E9C40EE66E000EE66ED9507E
:1006A000010FE66EDACFE6FFC40EE66E000EE66ED0
:1006B000C80EE66E710EE66EE66A600EE66E000E1D
:1006C000E66E80EC49F04BE9400EE66E600EE66E99
:1006D000000EE66E90EC1CF043E9000137510DE18D
:1006E000B30EE66E710EE66EE66A600EE66E000E02
:1006F000E66E80EC49F045E942D08DA234D000018D
:10070000060510E18B50100B0DE19E0EE66E710E8A
:10071000E66EE66A600EE66E000EE66E80EC49F06C
:1007200045E920D0020E0001065D10E18B50100B50
:100730000DE09E0EE66E710EE66EE66A600EE66EE7
:10074000000EE66E80EC49F045E90CD0890EE66EAD
:10075000710EE66EE66A600EE66E000EE66E80ECE6
:1007600049F045E90CD0890EE66E710EE66EE66A38
:10077000600EE66E000EE66E80EC49F045E9140E60
:10078000E66E600EE66E000EE66E90EC1CF043E93D
:100790008BA20DD0740EE66E710EE66EE66A600EE8
:1007A000E66E000EE66E80EC49F045E90CD05F0E77
:1007B000E66E710EE66EE66A600EE66E000EE66E9E
:1007C00080EC49F045E9540EE66E600EE66E000ED0
:1007D000E66E90EC1CF043E9DAEF1BF0030E00012B
:1007E000015D55E04A0EE66E710EE66EE66A600E39
:1007F000E66E000EE66E80EC49F045E9E66A600EB2
:10080000E66E000EE66E90EC1CF043E9350EE66EE7
:10081000710EE66EE66A600EE66E000EE66E80EC25
:1008200049F045E9400EE66E600EE66E000EE66E9B
:1008300090EC1CF043E9200EE66E710EE66EE66A5F
:10084000600EE66E000EE66E80EC49F045E9140E8F
:10085000E66E600EE66E000EE66E90EC1CF043E96C
:100860004A0EE66E710EE66EE66A600EE66E000EE9
:10087000E66E80EC49F045E9540EE66E600EE66ED9
:10088000000EE66E90EC1CF043E900C001F0DAEFD8
:100890001BF0040E0001015D55E04A0EE66E710E7C
:1008A000E66EE66A600EE66E000EE66E80EC49F0DB
:1008B00045E9E66A600EE66E000EE66E90EC1CF00E
:1008C00043E9350EE66E710EE66EE66A600EE66E80
:1008D000000EE66E80EC49F045E9400EE66E600ED3
:1008E000E66E000EE66E90EC1CF043E90B0EE66E31
:1008F000710EE66EE66A600EE66E000EE66E80EC45
:1009000049F045E9140EE66E600EE66E000EE66EE6
:1009100090EC1CF043E94A0EE66E710EE66EE66A54
:10092000600EE66E000EE66E80EC49F045E9540E6E
:10093000E66E600EE66E000EE66E90EC1CF043E98B
:1009400000C001F0DAEF1BF00A0E0001015D55E076
:100950004A0EE66E710EE66EE66A600EE66E000EF8
:10096000E66E80EC49F045E9E66A600EE66E000E40
:10097000E66E90EC1CF043E9F60EE66E700EE66E45
:10098000E66A600EE66E000EE66E80EC49F045E920
:10099000400EE66E600EE66E000EE66E90EC1CF009
:1009A00043E9E10EE66E700EE66EE66A600EE66EF4
:1009B000000EE66E80EC49F045E9140EE66E600E1E
:1009C000E66E000EE66E90EC1CF043E94A0EE66E11
:1009D000710EE66EE66A600EE66E000EE66E80EC64
:1009E00049F045E9540EE66E600EE66E000EE66EC6
:1009F00090EC1CF043E900C001F0DAEF1BF00B0EA5
:100A00000001015D55E04A0EE66E710EE66EE66A83
:100A1000600EE66E000EE66E80EC49F045E9E66A8F
:100A2000600EE66E000EE66E90EC1CF043E9F60EEA
:100A3000E66E700EE66EE66A600EE66E000EE66E1C
:100A400080EC49F045E9400EE66E600EE66E000E61
:100A5000E66E90EC1CF043E9CC0EE66E700EE66E8E
:100A6000E66A600EE66E000EE66E80EC49F045E93F
:100A7000140EE66E600EE66E000EE66E90EC1CF054
:100A800043E94A0EE66E710EE66EE66A600EE66EA9
:100A9000000EE66E80EC49F045E9540EE66E600EFD
:100AA000E66E000EE66E90EC1CF043E900C001F02B
:100AB000DAEF1BF00C0E0001015D55E04A0EE66E08
:100AC000710EE66EE66A600EE66E000EE66E80EC73
:100AD00049F045E9E66A600EE66E000EE66E90ECBF
:100AE0001CF043E9F60EE66E700EE66EE66A600EE6
:100AF000E66E000EE66E80EC49F045E9400EE66ECB
:100B0000600EE66E000EE66E90EC1CF043E9B70E48
:100B1000E66E700EE66EE66A600EE66E000EE66E3B
:100B200080EC49F045E9140EE66E600EE66E000EAC
:100B3000E66E90EC1CF043E94A0EE66E710EE66E2E
:100B4000E66A600EE66E000EE66E80EC49F045E95E
:100B5000540EE66E600EE66E000EE66E90EC1CF033
:100B600043E900C001F0DAEF1BF00D0E0001015D5A
:100B700055E04A0EE66E710EE66EE66A600EE66EAF
:100B8000000EE66E80EC49F045E9E66A600EE66E1E
:100B9000000EE66E90EC1CF043E9F60EE66E700E69
:100BA000E66EE66A600EE66E000EE66E80EC49F0D8
:100BB00045E9400EE66E600EE66E000EE66E90ECC5
:100BC0001CF043E9A20EE66E700EE66EE66A600E59
:100BD000E66E000EE66E80EC49F045E9140EE66E16
:100BE000600EE66E000EE66E90EC1CF043E94A0ED5
:100BF000E66E710EE66EE66A600EE66E000EE66E5A
:100C000080EC49F045E9540EE66E600EE66E000E8B
:100C1000E66E90EC1CF043E900C001F0DAEF1BF047
:100C20000E0E0001015D55E04A0EE66E710EE66E95
:100C3000E66A600EE66E000EE66E80EC49F045E96D
:100C4000E66A600EE66E000EE66E90EC1CF043E97C
:100C5000F60EE66E700EE66EE66A600EE66E000E4A
:100C6000E66E80EC49F045E9400EE66E600EE66EF9
:100C7000000EE66E90EC1CF043E98D0EE66E700EF1
:100C8000E66EE66A600EE66E000EE66E80EC49F0F7
:100C900045E9140EE66E600EE66E000EE66E90EC10
:100CA0001CF043E94A0EE66E710EE66EE66A600ECF
:100CB000E66E000EE66E80EC49F045E9540EE66EF5
:100CC000600EE66E000EE66E90EC1CF043E900C08C
:100CD00001F0DAEF1BF00F0E0001015D59E04A0E42
:100CE000E66E710EE66EE66A600EE66E000EE66E69
:100CF00080EC49F045E9E66A600EE66E000EE66EAD
:100D000090EC1CF043E9F60EE66E700EE66EE66AB5
:100D1000600EE66E000EE66E80EC49F045E9400E8E
:100D2000E66E600EE66E000EE66E90EC1CF043E997
:100D3000C40EE66E000EE66E770EE66E700EE66E80
:100D4000E66A600EE66E000EE66E80EC49F047E95A
:100D5000140EE66E600EE66E000EE66E90EC1CF071
:100D600043E94A0EE66E710EE66EE66A600EE66EC6
:100D7000000EE66E80EC49F045E9540EE66E600E1A
:100D8000E66E000EE66E90EC1CF043E900C001F048
:100D9000DAEF1BF0140E0001015D47E0620EE66E13
:100DA000700EE66EE66A600EE66E000EE66E80EC91
:100DB00049F045E9E66A600EE66E000EE66E90ECDC
:100DC0001CF043E9C60EE66E000EE66E5F0EE66EA0
:100DD000700EE66EE66A790EE66E000EE66E80EC48
:100DE00049F047E9C60EE66E000EE66E5F0EE66E4F
:100DF000700EE66EE66A920EE66E000EE66E80EC0F
:100E000049F047E9C60EE66E000EE66E5F0EE66E2E
:100E1000700EE66EE66AAB0EE66E000EE66E80ECD5
:100E200049F047E900C001F073D1000102511A0AEC
:100E300001E111D1030A01E1E3D0010A01E1BBD0D4
:100E40000F0A01E193D0010A6CE0030A2CE0010AC9
:100E500001E042D14A0EE66E700EE66EE66A790E49
:100E6000E66E000EE66E80EC49F045E9350EE66E62
:100E7000700EE66EE66A920EE66E000EE66E80EC8E
:100E800049F045E9C60EE66E000EE66E5F0EE66EB0
:100E9000700EE66EE66AAB0EE66E000EE66E80EC55
:100EA00049F047E91AD1200EE66E700EE66EE66A4A
:100EB000790EE66E000EE66E80EC49F045E90B0E09
:100EC000E66E700EE66EE66A920EE66E000EE66E56
:100ED00080EC49F045E9020E0001065D11E1C40E07
:100EE000E66E000EE66EF50EE66E6F0EE66EE66AD4
:100EF000AB0EE66E000EE66E80EC49F047E910D0CE
:100F0000C40EE66E000EE66EDF0EE66E6F0EE66E47
:100F1000E66AAB0EE66E000EE66E80EC49F047E93D
:100F2000DCD0200EE66E700EE66EE66A790EE66E96
:100F3000000EE66E80EC49F045E9CA0EE66E6F0ED3
:100F4000E66EE66A920EE66E000EE66E80EC49F002
:100F500045E9B50EE66E6F0EE66EE66AAB0EE66E1E
:100F6000000EE66E80EC49F045E9B7D0200EE66E43
:100F7000700EE66EE66A790EE66E000EE66E80ECA6
:100F800049F045E9A00EE66E6F0EE66EE66A920E37
:100F9000E66E000EE66E80EC49F045E98B0EE66EDB
:100FA0006F0EE66EE66AAB0EE66E000EE66E80EC45
:100FB00049F045E992D0200EE66E700EE66EE66AC4
:100FC000790EE66E000EE66E80EC49F045E9760E8D
:100FD000E66E6F0EE66EE66A920EE66E000EE66E46
:100FE00080EC49F045E9610EE66E6F0EE66EE66A4A
:100FF000AB0EE66E000EE66E80EC49F045E96DD072
:10100000200EE66E700EE66EE66A790EE66E000E53
:10101000E66E80EC49F045E94C0EE66E6F0EE66E2A
:10102000E66A920EE66E000EE66E80EC49F045E947
:10103000020EE66EE66A020EE66EE66A350EE66EB1
:101040006F0EE66EE66AAB0EE66E000EE66E80ECA4
:1010500049F049E942D0200EE66E6F0EE66EE66A70
:10106000790EE66E000EE66E80EC49F045E900016F
:10107000065119E10B0EE66E6F0EE66EE66A920EF1
:10108000E66E000EE66E80EC49F045E9F60EE66E7F
:101090006E0EE66EE66AAB0EE66E000EE66E80EC55
:1010A00049F045E918D0F60EE66E6E0EE66EE66A79
:1010B000920EE66E000EE66E80EC49F045E9E10E18
:1010C000E66E6E0EE66EE66AAB0EE66E000EE66E3D
:1010D00080EC49F045E901D000D0400EE66E790E73
:1010E000E66E000EE66E90EC1CF043E9140EE66E20
:1010F000920EE66E000EE66E90EC1CF043E9540E84
:10110000E66EAB0EE66E000EE66E90EC1CF043E968
:10111000DAEF1BF0150E0001015D4DE0CC0EE66E1E
:101120006E0EE66EE66A600EE66E000EE66E80EC0F
:1011300049F045E9E66A600EE66E000EE66E90EC58
:101140001CF043E9020E0001065D11E1C40EE66EDB
:10115000000EE66EB60EE66E6E0EE66EE66A600E87
:10116000E66E000EE66E80EC49F047E910D0C40E42
:10117000E66E000EE66EA00EE66E6E0EE66EE66A97
:10118000600EE66E000EE66E80EC49F047E9400E18
:10119000E66E600EE66E000EE66E90EC1CF043E923
:1011A000140EE66EC60EE66E000EE66E90EC1CF0B7
:1011B00043E900C001F004C0E6FF05C0E6FFD950D6
:1011C000010FE66EDACFE6FF05EC1DF044E9C40E30
:1011D000E66E000EE66ED950010FE66EDACFE6FF3E
:1011E0008D0EE66E6E0EE66EE66A600EE66E000E20
:1011F000E66E80EC49F049E9540EE66E600EE66E4C
:10120000000EE66E90EC1CF043E9DAEF1BF0160ED0
:101210000001015D34E0CC0EE66E6E0EE66EE66A0D
:10122000600EE66E000EE66E80EC49F045E9E66A77
:10123000600EE66E000EE66E90EC1CF043E9780E50
:10124000E66E6E0EE66EE66A600EE66E000EE66E06
:1012500080EC49F045E9400EE66E600EE66E000E49
:10126000E66E90EC1CF043E9140EE66EC60EE66ED8
:10127000000EE66E90EC1CF043E900C001F00001A6
:1012800002510DE1630EE66E6E0EE66EE66A600ECA
:10129000E66E000EE66E80EC49F045E92DD00001C7
:1012A00002050DE14E0EE66E6E0EE66EE66A600E0B
:1012B000E66E000EE66E80EC49F045E91DD0020EA8
:1012C0000001025D0DE1390EE66E6E0EE66EE66A15
:1012D000600EE66E000EE66E80EC49F045E90CD03B
:1012E000240EE66E6E0EE66EE66A600EE66E000E88
:1012F000E66E80EC49F045E9540EE66E600EE66E4F
:10130000000EE66E90EC1CF043E9DAEF1BF0170ECE
:101310000001015D34E0CC0EE66E6E0EE66EE66A0C
:10132000600EE66E000EE66E80EC49F045E9E66A76
:10133000600EE66E000EE66E90EC1CF043E90F0EB8
:10134000E66E6E0EE66EE66A600EE66E000EE66E05
:1013500080EC49F045E9400EE66E600EE66E000E48
:10136000E66E90EC1CF043E9140EE66EC60EE66ED7
:10137000000EE66E90EC1CF043E900C001F0020E96
:101380000001025D0DE1FA0EE66E6D0EE66EE66A94
:10139000600EE66E000EE66E80EC49F045E90FD077
:1013A000000102050CE1E50EE66E6D0EE66EE66AE2
:1013B000600EE66E000EE66E80EC49F045E9540ED4
:1013C000E66E600EE66E000EE66E90EC1CF043E9F1
:1013D000DAEF1BF0500E0001015D16E0D00EE66E54
:1013E0006D0EE66EE66A600EE66E000EE66E80EC4E
:1013F00049F045E9E66A600EE66E000EE66E90EC96
:101400001CF043E900C001F000010251580A01E15B
:101410004AD10F0A01E122D1010A01E1FAD0030AFF
:1014200001E1D2D0010A01E1A6D0070A01E17ED094
:10143000010A53E0030A2CE0010A01E059D14A0EE7
:10144000E66E700EE66EE66A790EE66E000EE66EE9
:1014500080EC49F045E9350EE66E700EE66EE66A00
:10146000920EE66E000EE66E80EC49F045E9C60E7F
:10147000E66E000EE66E5F0EE66E700EE66EE66AD3
:10148000AB0EE66E000EE66E80EC49F047E931D116
:10149000200EE66E700EE66EE66A790EE66E000EBF
:1014A000E66E80EC49F045E9BB0EE66E6D0EE66E29
:1014B000E66A920EE66E000EE66E80EC49F045E9B3
:1014C000A60EE66E6D0EE66EE66AAB0EE66E000EDA
:1014D000E66E80EC49F045E90CD1200EE66E700E08
:1014E000E66EE66A790EE66E000EE66E80EC49F076
:1014F00045E9910EE66E6D0EE66EE66A920EE66EB8
:10150000000EE66E80EC49F045E9C40EE66E000E72
:10151000E66E7C0EE66E6D0EE66EE66AAB0EE66E6D
:10152000000EE66E80EC49F047E9E3D0200EE66E4F
:10153000700EE66EE66A790EE66E000EE66E80ECE0
:1015400049F045E9670EE66E6D0EE66EE66A920EAC
:10155000E66E000EE66E80EC49F045E9520EE66E4E
:101560006D0EE66EE66AAB0EE66E000EE66E80EC81
:1015700049F045E9BED0200EE66E700EE66EE66AD2
:10158000790EE66E000EE66E80EC49F045E9670ED6
:10159000E66E6D0EE66EE66A920EE66E000EE66E82
:1015A00080EC49F045E9C40EE66E000EE66E3C0E96
:1015B000E66E6D0EE66EE66AAB0EE66E000EE66E49
:1015C00080EC49F047E995D0200EE66E700EE66E8D
:1015D000E66A790EE66E000EE66E80EC49F045E9AB
:1015E000910EE66E6D0EE66EE66A920EE66E000EE7
:1015F000E66E80EC49F045E9270EE66E6D0EE66E6C
:10160000E66AAB0EE66E000EE66E80EC49F045E948
:1016100070D0200EE66E700EE66EE66A790EE66E0B
:10162000000EE66E80EC49F045E9910EE66E6D0E17
:10163000E66EE66A920EE66E000EE66E80EC49F00B
:1016400045E9120EE66E6D0EE66EE66AAB0EE66ECC
:10165000000EE66E80EC49F045E94BD0200EE66EB8
:10166000700EE66EE66A790EE66E000EE66E80ECAF
:1016700049F045E9910EE66E6D0EE66EE66A920E51
:10168000E66E000EE66E80EC49F045E9FD0EE66E72
:101690006C0EE66EE66AAB0EE66E000EE66E80EC51
:1016A00049F045E926D0200EE66E6F0EE66EE66A3A
:1016B000790EE66E000EE66E80EC49F045E9E80E24
:1016C000E66E6C0EE66EE66A920EE66E000EE66E52
:1016D00080EC49F045E9D30EE66E6C0EE66EE66AE4
:1016E000AB0EE66E000EE66E80EC49F045E901D0E7
:1016F00000D0400EE66E790EE66E000EE66E90ECBF
:101700001CF043E9140EE66E920EE66E000EE66ED5
:1017100090EC1CF043E9540EE66EAB0EE66E000E44
:10172000E66E90EC1CF043E9DAEF1BF0510E00017D
:10173000015D17E0BE0EE66E6C0EE66EE66A600EA8
:10174000E66E000EE66E80EC49F045E9400EE66E6E
:10175000600EE66E000EE66E90EC1CF043E900C0F1
:1017600001F084A40DD0A90EE66E6C0EE66EE66A5A
:10177000600EE66E000EE66E80EC49F045E90CD096
:10178000940EE66E6C0EE66EE66A600EE66E000E75
:10179000E66E80EC49F045E9140EE66E600EE66EEA
:1017A000000EE66E90EC1CF043E984A00DD07F0E95
:1017B000E66E6C0EE66EE66A600EE66E000EE66E93
:1017C00080EC49F045E90CD06A0EE66E6C0EE66ED0
:1017D000E66A600EE66E000EE66E80EC49F045E9C2
:1017E000540EE66E600EE66E000EE66E90EC1CF097
:1017F00043E9DAEF1BF0520E0001015D30E0910E7B
:10180000E66E6D0EE66EE66A600EE66E000EE66E41
:1018100080EC49F045E9400EE66E600EE66E000E83
:10182000E66E90EC1CF043E9C40EE66E000EE66E28
:10183000550EE66E6C0EE66EE66A600EE66E000E03
:10184000E66E80EC49F047E9140EE66E600EE66E37
:10185000000EE66E90EC1CF043E900C001F08DA292
:101860000DD0400EE66E6C0EE66EE66A600EE66E19
:10187000000EE66E80EC49F045E90CD02B0EE66ECA
:101880006C0EE66EE66A600EE66E000EE66E80ECAA
:1018900049F045E9540EE66E600EE66E000EE66E07
:1018A00090EC1CF043E9DAEF1BF0530E0001015DF0
:1018B0002CE0670EE66E6D0EE66EE66A600EE66E72
:1018C000000EE66E80EC49F045E9400EE66E600ED3
:1018D000E66E000EE66E90EC1CF043E9520EE66EEA
:1018E0006D0EE66EE66A600EE66E000EE66E80EC49
:1018F00049F045E9140EE66E600EE66E000EE66EE7
:1019000090EC1CF043E900C001F08BA615D0C40E8A
:10191000E66E000EE66EC40EE66E000EE66E140E67
:10192000E66E6C0EE66EE66A600EE66E000EE66E21
:1019300080EC49F049E914D0C40EE66E000EE66E64
:10194000C40EE66E000EE66EFD0EE66E6B0EE66EE3
:10195000E66A600EE66E000EE66E80EC49F049E93C
:10196000540EE66E600EE66E000EE66E90EC1CF015
:1019700043E9DAEF1BF0540E0001015D30E0670E21
:10198000E66E6D0EE66EE66A600EE66E000EE66EC0
:1019900080EC49F045E9400EE66E600EE66E000E02
:1019A000E66E90EC1CF043E9C40EE66E000EE66EA7
:1019B000E70EE66E6B0EE66EE66A600EE66E000EF1
:1019C000E66E80EC49F047E9140EE66E600EE66EB6
:1019D000000EE66E90EC1CF043E900C001F08BA80D
:1019E00015D0C40EE66E000EE66EC40EE66E000E56
:1019F000E66ED00EE66E6B0EE66EE66A600EE66E82
:101A0000000EE66E80EC49F049E914D0C40EE66E93
:101A1000000EE66EC40EE66E000EE66EB90EE66EC1
:101A20006B0EE66EE66A600EE66E000EE66E80EC09
:101A300049F049E9540EE66E600EE66E000EE66E61
:101A400090EC1CF043E9DAEF1BF0550E0001015D4C
:101A50002CE0910EE66E6D0EE66EE66A600EE66EA6
:101A6000000EE66E80EC49F045E9400EE66E600E31
:101A7000E66E000EE66E90EC1CF043E9270EE66E73
:101A80006D0EE66EE66A600EE66E000EE66E80ECA7
:101A900049F045E9140EE66E600EE66E000EE66E45
:101AA00090EC1CF043E900C001F08BA40DD0400E77
:101AB000E66E6C0EE66EE66A600EE66E000EE66E90
:101AC00080EC49F045E90CD02B0EE66E6C0EE66E0C
:101AD000E66A600EE66E000EE66E80EC49F045E9BF
:101AE000540EE66E600EE66E000EE66E90EC1CF094
:101AF00043E9DAEF1BF0560E0001015D2CE0910E78
:101B0000E66E6D0EE66EE66A600EE66E000EE66E3E
:101B100080EC49F045E9400EE66E600EE66E000E80
:101B2000E66E90EC1CF043E9120EE66E6D0EE66E6A
:101B3000E66A600EE66E000EE66E80EC49F045E95E
:101B4000140EE66E600EE66E000EE66E90EC1CF073
:101B500043E900C001F08BA20DD0400EE66E6C0E82
:101B6000E66EE66A600EE66E000EE66E80EC49F008
:101B700045E90CD02B0EE66E6C0EE66EE66A600E42
:101B8000E66E000EE66E80EC49F045E9540EE66E16
:101B9000600EE66E000EE66E90EC1CF043E9DAEFA4
:101BA0001BF0570E0001015D2CE0910EE66E6D0EEC
:101BB000E66EE66A600EE66E000EE66E80EC49F0B8
:101BC00045E9400EE66E600EE66E000EE66E90ECA5
:101BD0001CF043E9FD0EE66E6C0EE66EE66A600EE2
:101BE000E66E000EE66E80EC49F045E9140EE66EF6
:101BF000600EE66E000EE66E90EC1CF043E900C04D
:101C000001F08BA00DD0400EE66E6C0EE66EE66A1B
:101C1000600EE66E000EE66E80EC49F045E90CD0F1
:101C20002B0EE66E6C0EE66EE66A600EE66E000E39
:101C3000E66E80EC49F045E9540EE66E600EE66E05
:101C4000000EE66E90EC1CF043E9DAEF1BF0580E44
:101C50000001015D2CE0E80EE66E6C0EE66EE66AB1
:101C6000600EE66E000EE66E80EC49F045E9400E2F
:101C7000E66E600EE66E000EE66E90EC1CF043E938
:101C8000D30EE66E6C0EE66EE66A600EE66E000E31
:101C9000E66E80EC49F045E9140EE66E600EE66EE5
:101CA000000EE66E90EC1CF043E900C001F0895094
:101CB000400B10E08950800B0DE1A40EE66E6B0E18
:101CC000E66EE66A600EE66E000EE66E80EC49F0A7
:101CD00045E932D08950400B10E18950800B0DE06E
:101CE0008F0EE66E6B0EE66EE66A600EE66E000E16
:101CF000E66E80EC49F045E91FD08950400B10E1B9
:101D00008950800B0DE17A0EE66E6B0EE66EE66A88
:101D1000600EE66E000EE66E80EC49F045E90CD0F0
:101D2000650EE66E6B0EE66EE66A600EE66E000EFF
:101D3000E66E80EC49F045E9540EE66E600EE66E04
:101D4000000EE66E90EC1CF043E9DAEF1BF0280E73
:101D50000001015D16E0500EE66E6B0EE66EE66A5F
:101D6000600EE66E000EE66E80EC49F045E9E66A2C
:101D7000600EE66E000EE66E90EC1CF043E900C0CB
:101D800001F000010251370A01E16AD2010A01E1C2
:101D900042D2030A01E11AD2010A01E1F2D1070A93
:101DA00001E1C6D1010A01E19AD1030A01E172D130
:101DB000010A01E14AD11F0A01E122D1010A01E130
:101DC000FAD0030A01E1D2D0010A01E1AAD0070A40
:101DD00001E182D0010A57E0030A2CE0010A01E088
:101DE00064D24A0EE66E700EE66EE66A790EE66E14
:101DF000000EE66E80EC49F045E9350EE66E700E99
:101E0000E66EE66A920EE66E000EE66E80EC49F033
:101E100045E9C60EE66E000EE66E5F0EE66E700ECB
:101E2000E66EE66AAB0EE66E000EE66E80EC49F0FA
:101E300047E93CD2200EE66E700EE66EE66A790E39
:101E4000E66E000EE66E80EC49F045E93B0EE66E6C
:101E50006B0EE66EE66A920EE66E000EE66E80ECA3
:101E600049F045E9C60EE66E000EE66E5F0EE66EC0
:101E7000700EE66EE66AAB0EE66E000EE66E80EC65
:101E800049F047E913D2200EE66E700EE66EE66A60
:101E9000790EE66E000EE66E80EC49F045E9260EFE
:101EA000E66E6B0EE66EE66A920EE66E000EE66E6B
:101EB00080EC49F045E9C60EE66E000EE66E5F0E58
:101EC000E66E700EE66EE66AAB0EE66E000EE66E2D
:101ED00080EC49F047E9EAD1200EE66E700EE66E1E
:101EE000E66A790EE66E000EE66E80EC49F045E992
:101EF000110EE66E6B0EE66EE66A920EE66E000E50
:101F0000E66E80EC49F045E9FC0EE66E6A0EE66E80
:101F1000E66AAB0EE66E000EE66E80EC49F045E92F
:101F2000C5D1200EE66E700EE66EE66A790EE66E9C
:101F3000000EE66E80EC49F045E9110EE66E6B0E80
:101F4000E66EE66A920EE66E000EE66E80EC49F0F2
:101F500045E9E70EE66E6A0EE66EE66AAB0EE66EE1
:101F6000000EE66E80EC49F045E9A0D1200EE66E49
:101F7000700EE66EE66A790EE66E000EE66E80EC96
:101F800049F045E9D20EE66E6A0EE66EE66A920EFA
:101F9000E66E000EE66E80EC49F045E9BD0EE66E99
:101FA0006A0EE66EE66AAB0EE66E000EE66E80EC3A
:101FB00049F045E97BD1200EE66E700EE66EE66ACA
:101FC000790EE66E000EE66E80EC49F045E9A80E4B
:101FD000E66E6A0EE66EE66A920EE66E000EE66E3B
:101FE00080EC49F045E9930EE66E6A0EE66EE66A0D
:101FF000AB0EE66E000EE66E80EC49F045E956D178
:10200000200EE66E700EE66EE66A790EE66E000E43
:10201000E66E80EC49F045E97E0EE66E6A0EE66EED
:10202000E66A920EE66E000EE66E80EC49F045E937
:10203000690EE66E6A0EE66EE66AAB0EE66E000E9E
:10204000E66E80EC49F045E931D1200EE66E700E67
:10205000E66EE66A790EE66E000EE66E80EC49F0FA
:1020600045E97E0EE66E6A0EE66EE66A920EE66E52
:10207000000EE66E80EC49F045E9540EE66E6A0EFD
:10208000E66EE66AAB0EE66E000EE66E80EC49F098
:1020900045E90CD1200EE66E700EE66EE66A790E0A
:1020A000E66E000EE66E80EC49F045E93F0EE66E06
:1020B0006A0EE66EE66A920EE66E000EE66E80EC42
:1020C00049F045E92A0EE66E6A0EE66EE66AAB0E48
:1020D000E66E000EE66E80EC49F045E9E7D0200E92
:1020E000E66E700EE66EE66A790EE66E000EE66E3D
:1020F00080EC49F045E9C40EE66E000EE66E140E63
:10210000E66E6A0EE66EE66A920EE66E000EE66E09
:1021100080EC49F047E9FF0EE66E690EE66EE66A6E
:10212000AB0EE66E000EE66E80EC49F045E9BED0DF
:10213000200EE66E700EE66EE66A790EE66E000E12
:10214000E66E80EC49F045E9C40EE66E000EE66EE0
:10215000140EE66E6A0EE66EE66A920EE66E000EEB
:10216000E66E80EC49F047E9EA0EE66E690EE66E2F
:10217000E66AAB0EE66E000EE66E80EC49F045E9CD
:1021800095D0200EE66E700EE66EE66A790EE66E6B
:10219000000EE66E80EC49F045E9D50EE66E690E5C
:1021A000E66EE66A920EE66E000EE66E80EC49F090
:1021B00045E9C00EE66E690EE66EE66AAB0EE66EA7
:1021C000000EE66E80EC49F045E970D0200EE66E18
:1021D000700EE66EE66A790EE66E000EE66E80EC34
:1021E00049F045E9AB0EE66E690EE66EE66A920EC0
:1021F000E66E000EE66E80EC49F045E9960EE66E5E
:10220000690EE66EE66AAB0EE66E000EE66E80ECD8
:1022100049F045E94BD0200EE66E700EE66EE66A98
:10222000790EE66E000EE66E80EC49F045E9AB0EE5
:10223000E66E690EE66EE66A920EE66E000EE66ED9
:1022400080EC49F045E9810EE66E690EE66EE66ABD
:10225000AB0EE66E000EE66E80EC49F045E926D046
:10226000200EE66E6F0EE66EE66A790EE66E000EE2
:10227000E66E80EC49F045E96C0EE66E690EE66E9E
:10228000E66A920EE66E000EE66E80EC49F045E9D5
:10229000570EE66E690EE66EE66AAB0EE66E000E4F
:1022A000E66E80EC49F045E901D000D0400EE66EC4
:1022B000790EE66E000EE66E90EC1CF043E9140E0B
:1022C000E66E920EE66E000EE66E90EC1CF043E9B0
:1022D000540EE66EAB0EE66E000EE66E90EC1CF051
:1022E00043E9DAEF1BF0290E0001015D20E03B0E0F
:1022F000E66E6B0EE66EE66A600EE66E000EE66E49
:1023000080EC49F045E9400EE66E600EE66E000E88
:10231000E66E90EC1CF043E9140EE66EC60EE66E17
:10232000000EE66E90EC1CF043E900C001F004C022
:10233000E6FF05C0E6FFD950010FE66EDACFE6FFF3
:1023400005EC1DF044E9D950010FE66EDACFE6FF47
:10235000440EE66E690EE66EE66A600EE66E000EEC
:10236000E66E80EC49F047E9540EE66E600EE66ECC
:10237000000EE66E90EC1CF043E9DAEF1BF02A0E3B
:102380000001015D30E0260EE66E6B0EE66EE66A39
:10239000600EE66E000EE66E80EC49F045E9400EF8
:1023A000E66E600EE66E000EE66E90EC1CF043E901
:1023B000C40EE66E000EE66E2E0EE66E690EE66E3A
:1023C000E66A600EE66E000EE66E80EC49F047E9C4
:1023D000140EE66E600EE66E000EE66E90EC1CF0DB
:1023E00043E900C001F004C0E6FF05C0E6FFD95094
:1023F000010FE66EDACFE6FF05EC1DF044E9C40EEE
:10240000E66E000EE66ED950010FE66EDACFE6FFFB
:102410008D0EE66E6E0EE66EE66A600EE66E000EDD
:10242000E66E80EC49F049E9540EE66E600EE66E09
:10243000000EE66E90EC1CF043E9DAEF1BF02B0E79
:102440000001015D2CE0110EE66E6B0EE66EE66A91
:10245000600EE66E000EE66E80EC49F045E9400E37
:10246000E66E600EE66E000EE66E90EC1CF043E940
:10247000FC0EE66E6A0EE66EE66A600EE66E000E12
:10248000E66E80EC49F045E9140EE66E600EE66EED
:10249000000EE66E90EC1CF043E900C001F004C0B1
:1024A000E6FF05C0E6FFD950010FE66EDACFE6FF82
:1024B00005EC1DF044E9C40EE66E000EE66ED95040
:1024C000010FE66EDACFE6FF8D0EE66E6E0EE66E5B
:1024D000E66A600EE66E000EE66E80EC49F049E9B1
:1024E000540EE66E600EE66E000EE66E90EC1CF08A
:1024F00043E9DAEF1BF02C0E0001015D2CE0110E18
:10250000E66E6B0EE66EE66A600EE66E000EE66E36
:1025100080EC49F045E9400EE66E600EE66E000E76
:10252000E66E90EC1CF043E9E70EE66E6A0EE66E8E
:10253000E66A600EE66E000EE66E80EC49F045E954
:10254000140EE66E600EE66E000EE66E90EC1CF069
:1025500043E900C001F004C0E6FF05C0E6FFD95022
:10256000010FE66EDACFE6FF05EC1DF044E9C40E7C
:10257000E66E000EE66ED950010FE66EDACFE6FF8A
:102580008D0EE66E6E0EE66EE66A600EE66E000E6C
:10259000E66E80EC49F049E9540EE66E600EE66E98
:1025A000000EE66E90EC1CF043E9DAEF1BF02D0E06
:1025B0000001015D2CE0D20EE66E6A0EE66EE66A60
:1025C000600EE66E000EE66E80EC49F045E9400EC6
:1025D000E66E600EE66E000EE66E90EC1CF043E9CF
:1025E000BD0EE66E6A0EE66EE66A600EE66E000EE0
:1025F000E66E80EC49F045E9140EE66E600EE66E7C
:10260000000EE66E90EC1CF043E900C001F004C03F
:10261000E6FF05C0E6FFD950010FE66EDACFE6FF10
:1026200005EC1DF044E9C40EE66E000EE66ED950CE
:10263000010FE66EDACFE6FF8D0EE66E6E0EE66EE9
:10264000E66A600EE66E000EE66E80EC49F049E93F
:10265000540EE66E600EE66E000EE66E90EC1CF018
:1026600043E9DAEF1BF02E0E0001015D2CE0A80E0D
:10267000E66E6A0EE66EE66A600EE66E000EE66EC6
:1026800080EC49F045E9400EE66E600EE66E000E05
:10269000E66E90EC1CF043E9930EE66E6A0EE66E71
:1026A000E66A600EE66E000EE66E80EC49F045E9E3
:1026B000140EE66E600EE66E000EE66E90EC1CF0F8
:1026C00043E900C001F004C0E6FF05C0E6FFD950B1
:1026D000010FE66EDACFE6FF05EC1DF044E9C40E0B
:1026E000E66E000EE66ED950010FE66EDACFE6FF19
:1026F0008D0EE66E6E0EE66EE66A600EE66E000EFB
:10270000E66E80EC49F049E9540EE66E600EE66E26
:10271000000EE66E90EC1CF043E9DAEF1BF02F0E92
:102720000001015D2CE07E0EE66E6A0EE66EE66A42
:10273000600EE66E000EE66E80EC49F045E9400E54
:10274000E66E600EE66E000EE66E90EC1CF043E95D
:10275000690EE66E6A0EE66EE66A600EE66E000EC2
:10276000E66E80EC49F045E9140EE66E600EE66E0A
:10277000000EE66E90EC1CF043E900C001F004C0CE
:10278000E6FF05C0E6FFD950010FE66EDACFE6FF9F
:1027900005EC1DF044E9D950010FE66EDACFE6FFF3
:1027A0001C0EE66E690EE66EE66A600EE66E000EC0
:1027B000E66E80EC49F047E9540EE66E600EE66E78
:1027C000000EE66E90EC1CF043E9DAEF1BF0300EE1
:1027D0000001015D2CE07E0EE66E6A0EE66EE66A92
:1027E000600EE66E000EE66E80EC49F045E9400EA4
:1027F000E66E600EE66E000EE66E90EC1CF043E9AD
:10280000540EE66E6A0EE66EE66A600EE66E000E26
:10281000E66E80EC49F045E9140EE66E600EE66E59
:10282000000EE66E90EC1CF043E900C001F004C01D
:10283000E6FF05C0E6FFD950010FE66EDACFE6FFEE
:1028400005EC1DF044E9D950010FE66EDACFE6FF42
:102850001C0EE66E690EE66EE66A600EE66E000E0F
:10286000E66E80EC49F047E9540EE66E600EE66EC7
:10287000000EE66E90EC1CF043E9DAEF1BF0310E2F
:102880000001015D2CE03F0EE66E6A0EE66EE66A20
:10289000600EE66E000EE66E80EC49F045E9400EF3
:1028A000E66E600EE66E000EE66E90EC1CF043E9FC
:1028B0002A0EE66E6A0EE66EE66A600EE66E000EA0
:1028C000E66E80EC49F045E9140EE66E600EE66EA9
:1028D000000EE66E90EC1CF043E900C001F004C06D
:1028E000E6FF05C0E6FFD950010FE66EDACFE6FF3E
:1028F00005EC1DF044E9D950010FE66EDACFE6FF92
:102900001C0EE66E690EE66EE66A600EE66E000E5E
:10291000E66E80EC49F047E9540EE66E600EE66E16
:10292000000EE66E90EC1CF043E9DAEF1BF0320E7D
:102930000001015D30E0C40EE66E000EE66E140E7E
:10294000E66E6A0EE66EE66A600EE66E000EE66EF3
:1029500080EC49F047E9400EE66E600EE66E000E30
:10296000E66E90EC1CF043E9FF0EE66E690EE66E33
:10297000E66A600EE66E000EE66E80EC49F045E910
:10298000140EE66E600EE66E000EE66E90EC1CF025
:1029900043E900C001F004C0E6FF05C0E6FFD950DE
:1029A000010FE66EDACFE6FF05EC1DF044E9C40E38
:1029B000E66E000EE66ED950010FE66EDACFE6FF46
:1029C0008D0EE66E6E0EE66EE66A600EE66E000E28
:1029D000E66E80EC49F049E9540EE66E600EE66E54
:1029E000000EE66E90EC1CF043E9DAEF1BF0330EBC
:1029F0000001015D30E0C40EE66E000EE66E140EBE
:102A0000E66E6A0EE66EE66A600EE66E000EE66E32
:102A100080EC49F047E9400EE66E600EE66E000E6F
:102A2000E66E90EC1CF043E9EA0EE66E690EE66E87
:102A3000E66A600EE66E000EE66E80EC49F045E94F
:102A4000140EE66E600EE66E000EE66E90EC1CF064
:102A500043E900C001F004C0E6FF05C0E6FFD9501D
:102A6000010FE66EDACFE6FF05EC1DF044E9C40E77
:102A7000E66E000EE66ED950010FE66EDACFE6FF85
:102A80008D0EE66E6E0EE66EE66A600EE66E000E67
:102A9000E66E80EC49F049E9540EE66E600EE66E93
:102AA000000EE66E90EC1CF043E9DAEF1BF0340EFA
:102AB0000001015D2CE0D50EE66E690EE66EE66A59
:102AC000600EE66E000EE66E80EC49F045E9400EC1
:102AD000E66E600EE66E000EE66E90EC1CF043E9CA
:102AE000C00EE66E690EE66EE66A600EE66E000ED9
:102AF000E66E80EC49F045E9140EE66E600EE66E77
:102B0000000EE66E90EC1CF043E900C001F00001FD
:102B1000020E041901E105510DE1070EE66E690E82
:102B2000E66EE66A600EE66E000EE66E80EC49F038
:102B300045E91FD00001010E041901E105510DE125
:102B4000F20EE66E680EE66EE66A600EE66E000E47
:102B5000E66E80EC49F045E90CD0DD0EE66E680EBD
:102B6000E66EE66A600EE66E000EE66E80EC49F0F8
:102B700045E9540EE66E600EE66E000EE66E90ECD1
:102B80001CF043E9DAEF1BF0350E0001015D2CE08B
:102B9000AB0EE66E690EE66EE66A600EE66E000E3D
:102BA000E66E80EC49F045E9400EE66E600EE66E9A
:102BB000000EE66E90EC1CF043E9960EE66E690E90
:102BC000E66EE66A600EE66E000EE66E80EC49F098
:102BD00045E9140EE66E600EE66E000EE66E90ECB1
:102BE0001CF043E900C001F004C0E6FF05C0E6FFA9
:102BF000D950010FE66EDACFE6FF05EC1DF044E98F
:102C0000C40EE66E000EE66ED950010FE66EDACF06
:102C1000E6FF8D0EE66E6E0EE66EE66A600EE66EFE
:102C2000000EE66E80EC49F049E9540EE66E600E47
:102C3000E66E000EE66E90EC1CF043E9DAEF1BF056
:102C4000360E0001015D2CE0AB0EE66E690EE66EFD
:102C5000E66A600EE66E000EE66E80EC49F045E92D
:102C6000400EE66E600EE66E000EE66E90EC1CF016
:102C700043E9810EE66E690EE66EE66A600EE66E68
:102C8000000EE66E80EC49F045E9140EE66E600E2B
:102C9000E66E000EE66E90EC1CF043E900C001F019
:102CA00004C0E6FF05C0E6FFD950010FE66EDACF9B
:102CB000E6FF05EC1DF044E9C40EE66E000EE66E7C
:102CC000D950010FE66EDACFE6FF8D0EE66E6E0E7E
:102CD000E66EE66A600EE66E000EE66E80EC49F087
:102CE00049E9540EE66E600EE66E000EE66E90EC5C
:102CF0001CF043E9DAEF1BF0370E0001015D2CE018
:102D00006C0EE66E690EE66EE66A600EE66E000E0A
:102D1000E66E80EC49F045E9400EE66E600EE66E28
:102D2000000EE66E90EC1CF043E9570EE66E690E5D
:102D3000E66EE66A600EE66E000EE66E80EC49F026
:102D400045E9140EE66E600EE66E000EE66E90EC3F
:102D50001CF043E900C001F004C0E6FF05C0E6FF37
:102D6000D950010FE66EDACFE6FF05EC1DF044E91D
:102D7000C40EE66E000EE66ED950010FE66EDACF95
:102D8000E6FF8D0EE66E6E0EE66EE66A600EE66E8D
:102D9000000EE66E80EC49F049E9540EE66E600ED6
:102DA000E66E000EE66E90EC1CF043E9DAEF1BF0E5
:102DB000640E0001015D4BE0C80EE66E680EE66E23
:102DC000E66A600EE66E000EE66E80EC49F045E9BC
:102DD000E66A600EE66E000EE66E90EC1CF043E9CB
:102DE000400EE66EC60EE66E000EE66E90EC1CF02F
:102DF00043E9B30EE66E680EE66EE66A600EE66EB6
:102E0000000EE66E80EC49F045E9140EE66E600EA9
:102E1000E66E000EE66E90EC1CF043E99E0EE66E48
:102E2000680EE66EE66A600EE66E000EE66E80ECF8
:102E300049F045E9540EE66E600EE66E000EE66E51
:102E400090EC1CF043E900C001F081A4FED7000122
:102E50000251680A01E10BD10F0A01E1C4D0010A55
:102E600001E17DD0030A37E0010A01E044D14A0EB6
:102E7000E66E700EE66EE66A600EE66E000EE66EB8
:102E800080EC49F045E9400EE66E600EE66E000EFD
:102E9000E66E90EC1CF043E9350EE66E700EE66EC1
:102EA000E66A600EE66E000EE66E80EC49F045E9DB
:102EB000140EE66E600EE66E000EE66E90EC1CF0F0
:102EC00043E9540EE66EC60EE66E000EE66E90EC1A
:102ED0001CF043E911D1200EE66E700EE66EE66A34
:102EE000600EE66E000EE66E80EC49F045E9400E9D
:102EF000E66E600EE66E000EE66E90EC1CF043E9A6
:102F0000C40EE66E000EE66E890EE66E680EE66E84
:102F1000E66A600EE66E000EE66E80EC49F047E968
:102F2000140EE66E600EE66E000EE66E90EC1CF07F
:102F300043E9740EE66E680EE66EE66A600EE66EB3
:102F4000000EE66E80EC49F045E9540EE66E600E28
:102F5000E66E000EE66E90EC1CF043E9CDD0200E3C
:102F6000E66E700EE66EE66A600EE66E000EE66EC7
:102F700080EC49F045E9400EE66E600EE66E000E0C
:102F8000E66E90EC1CF043E9C40EE66E000EE66EB1
:102F9000890EE66E680EE66EE66A600EE66E000E5C
:102FA000E66E80EC49F047E9140EE66E600EE66EC0
:102FB000000EE66E90EC1CF043E95F0EE66E680EC4
:102FC000E66EE66A600EE66E000EE66E80EC49F094
:102FD00045E9540EE66E600EE66E000EE66E90EC6D
:102FE0001CF043E989D0200EE66E700EE66EE66AAC
:102FF000600EE66E000EE66E80EC49F045E9400E8C
:10300000E66E600EE66E000EE66E90EC1CF043E994
:10301000C40EE66E000EE66E890EE66E680EE66E73
:10302000E66A600EE66E000EE66E80EC49F047E957
:10303000140EE66E600EE66E000EE66E90EC1CF06E
:1030400043E94A0EE66E680EE66EE66A600EE66ECC
:10305000000EE66E80EC49F045E9540EE66E600E17
:10306000E66E000EE66E90EC1CF043E945D0200EB3
:10307000E66E6F0EE66EE66A600EE66E000EE66EB7
:1030800080EC49F045E9400EE66E600EE66E000EFB
:10309000E66E90EC1CF043E9C40EE66E000EE66EA0
:1030A000890EE66E680EE66EE66A600EE66E000E4B
:1030B000E66E80EC49F047E9140EE66E600EE66EAF
:1030C000000EE66E90EC1CF043E9350EE66E680EDD
:1030D000E66EE66A600EE66E000EE66E80EC49F083
:1030E00045E9540EE66E600EE66E000EE66E90EC5C
:1030F0001CF043E901D000D05DD3650E0001015DF5
:1031000022E0C40EE66E000EE66E200EE66E680E3D
:10311000E66EE66A600EE66E000EE66E80EC49F042
:1031200047E9400EE66E600EE66E000EE66EF8DBD6
:1031300043E9140EE66EC60EE66E000EE66EF0DB98
:1031400043E900C001F0700E00011F1902E1170EE3
:10315000201931E1C40EE66E000EE66E0B0EE66E2F
:10316000680EE66EE66A600EE66E000EE66E80ECB5
:1031700049F047E9140EE66E600EE66E000EE66E4C
:10318000CFDB43E9C40EE66E000EE66EF60EE66E89
:10319000670EE66EE66A600EE66E000EE66E80EC86
:1031A00049F047E9540EE66E600EE66E000EE66EDC
:1031B000B7DB43E978D0880E00011F1902E1130E36
:1031C000201931E1C40EE66E000EE66EE10EE66EE9
:1031D000670EE66EE66A600EE66E000EE66E80EC46
:1031E00049F047E9140EE66E600EE66E000EE66EDC
:1031F00097DB43E9C40EE66E000EE66ECC0EE66E7B
:10320000670EE66EE66A600EE66E000EE66E80EC15
:1032100049F047E9540EE66E600EE66E000EE66E6B
:103220007FDB43E940D01FC0E6FF20C0E6FFBA0EB7
:10323000E66E670EE66EE66A600EE66E000EE66EFD
:1032400080EC49F047E9140EE66E600EE66E000E63
:10325000E66E66DB43E921C0E6FF22C0E6FFD950F7
:10326000010FE66EDACFE6FFD0DB44E9C40EE66E6E
:10327000000EE66ED950010FE66EDACFE6FFA60E1D
:10328000E66E670EE66EE66A600EE66E000EE66EAD
:1032900080EC49F049E9540EE66E600EE66E000ED1
:1032A000E66E3EDB43E986D2660E0001015D22E058
:1032B000C40EE66E000EE66E910EE66E670EE66ECA
:1032C000E66A600EE66E000EE66E80EC49F047E9B5
:1032D000400EE66E600EE66E000EE66E21DB43E900
:1032E000140EE66EC60EE66E000EE66E19DB43E9BE
:1032F00000C001F0700E0001251902E1170E261919
:1033000031E1C40EE66E000EE66E0B0EE66E680E40
:10331000E66EE66A600EE66E000EE66E80EC49F040
:1033200047E9140EE66E600EE66E000EE66EF8DA01
:1033300043E9C40EE66E000EE66EF60EE66E670E0C
:10334000E66EE66A600EE66E000EE66E80EC49F010
:1033500047E9540EE66E600EE66E000EE66EE0DAA9
:1033600043E978D0880E0001251902E1130E2619D1
:1033700031E1C40EE66E000EE66EE10EE66E670EFB
:10338000E66EE66A600EE66E000EE66E80EC49F0D0
:1033900047E9140EE66E600EE66E000EE66EC0DAC9
:1033A00043E9C40EE66E000EE66ECC0EE66E670EC6
:1033B000E66EE66A600EE66E000EE66E80EC49F0A0
:1033C00047E9540EE66E600EE66E000EE66EA8DA71
:1033D00043E940D025C0E6FF26C0E6FFBA0EE66E00
:1033E000670EE66EE66A600EE66E000EE66E80EC34
:1033F00049F047E9140EE66E600EE66E000EE66ECA
:103400008FDA43E927C0E6FF28C0E6FFD950010F55
:10341000E66EDACFE6FFF9DA44E9C40EE66E000E96
:10342000E66ED950010FE66EDACFE6FFA60EE66E25
:10343000670EE66EE66A600EE66E000EE66E80ECE3
:1034400049F049E9540EE66E600EE66E000EE66E37
:1034500067DA43E9AFD1670E0001015D22E0C40ED7
:10346000E66E000EE66E7C0EE66E670EE66EE66AAF
:10347000600EE66E000EE66E80EC49F047E9400E05
:10348000E66E600EE66E000EE66E4ADA43E9140E52
:10349000E66EC60EE66E000EE66E42DA43E900C046
:1034A00001F0700E00012B1902E1170E2C1931E109
:1034B000C40EE66E000EE66E0B0EE66E680EE66E4D
:1034C000E66A600EE66E000EE66E80EC49F047E9B3
:1034D000140EE66E600EE66E000EE66E21DA43E92B
:1034E000C40EE66E000EE66EF60EE66E670EE66E33
:1034F000E66A600EE66E000EE66E80EC49F047E983
:10350000540EE66E600EE66E000EE66E09DA43E9D2
:1035100078D0880E00012B1902E1130E2C1931E12D
:10352000C40EE66E000EE66EE10EE66E670EE66E07
:10353000E66A600EE66E000EE66E80EC49F047E942
:10354000140EE66E600EE66E000EE66EE9D943E9F3
:10355000C40EE66E000EE66ECC0EE66E670EE66EEC
:10356000E66A600EE66E000EE66E80EC49F047E912
:10357000540EE66E600EE66E000EE66ED1D943E99B
:1035800040D02BC0E6FF2CC0E6FFBA0EE66E670EF9
:10359000E66EE66A600EE66E000EE66E80EC49F0BE
:1035A00047E9140EE66E600EE66E000EE66EB8D9C0
:1035B00043E92DC0E6FF2EC0E6FFD950010FE66EAD
:1035C000DACFE6FF22DA44E9C40EE66E000EE66EBC
:1035D000D950010FE66EDACFE6FFA60EE66E670E53
:1035E000E66EE66A600EE66E000EE66E80EC49F06E
:1035F00049E9540EE66E600EE66E000EE66E90D956
:1036000043E9D8D0680E0001015D22E0C40EE66EE9
:10361000000EE66E670EE66E670EE66EE66A600EF8
:10362000E66E000EE66E80EC49F047E9400EE66E6D
:10363000600EE66E000EE66E73D943E9140EE66E78
:10364000C60EE66E000EE66E6BD943E900C001F0CF
:10365000700E0001311902E1170E321931E1C40E6A
:10366000E66E000EE66E0B0EE66E680EE66EE66A1D
:10367000600EE66E000EE66E80EC49F047E9140E2F
:10368000E66E600EE66E000EE66E4AD943E9C40EA1
:10369000E66E000EE66EF60EE66E670EE66EE66A03
:1036A000600EE66E000EE66E80EC49F047E9540EBF
:1036B000E66E600EE66E000EE66E32D943E978D013
:1036C000880E0001311902E1130E321931E1C40EE6
:1036D000E66E000EE66EE10EE66E670EE66EE66AD8
:1036E000600EE66E000EE66E80EC49F047E9140EBF
:1036F000E66E600EE66E000EE66E12D943E9C40E69
:10370000E66E000EE66ECC0EE66E670EE66EE66ABC
:10371000600EE66E000EE66E80EC49F047E9540E4E
:10372000E66E600EE66E000EE66EFAD843E940D013
:1037300031C0E6FF32C0E6FFBA0EE66E670EE66EF7
:10374000E66A600EE66E000EE66E80EC49F047E930
:10375000140EE66E600EE66E000EE66EE1D843E9EA
:1037600033C0E6FF34C0E6FFD950010FE66EDACF72
:10377000E6FF4BD944E9C40EE66E000EE66ED95062
:10378000010FE66EDACFE6FFA60EE66E670EE66E76
:10379000E66A600EE66E000EE66E80EC49F049E9DE
:1037A000540EE66E600EE66E000EE66EB9D843E982
:1037B00001D000D00001005107E00001000504E045
:1037C000020E0001005D36E1020E00013D5D07E1E1
:1037D000130EE66E4F0EE66EBDD842E911D0030E11
:1037E00000013D5D07E1130EE66E460EE66EB2D8AF
:1037F00042E906D0130EE66E2D0EE66EABD842E916
:103800000001385103E0000137510FE100010305C9
:1038100006E1E66A450EE66E9DD842E905D0E66A05
:10382000200EE66E97D842E905D0E66A2D0EE66EC8
:1038300091D842E947E9E7CFD9FF1200D9CFE6FF97
:10384000E1CFD9FF81E959E8520EE66E670EE66EC8
:10385000E66AD950010FE66EDACFE6FF80EC49F058
:1038600045E9E66AD950010FE66EDACFE6FF58D88F
:1038700043E93D0EE66E670EE66EE66AD950010F2B
:10388000E66EDACFE6FF80EC49F045E9400EE66EE1
:10389000D950010FE66EDACFE6FF42D843E94A0E6F
:1038A000E66E710EE66EE66AD950010FE66EDACF6B
:1038B000E6FF80EC49F045E9140EE66ED950010FA1
:1038C000E66EDACFE6FF2CD843E9020EE66EE66A32
:1038D000020EE66EE66A260EE66E670EE66EE66A93
:1038E000D950010FE66EDACFE6FF80EC49F049E9E6
:1038F000540EE66ED950010FE66EDACFE6FF10D80F
:1039000043E95AE9E7CFD9FF1200E7EC4BF0000991
:1039100001E0FBD7010EE66E71EC4BF041E91200BD
:10392000D9CFE6FFE1CFD9FF84E9E7EC4BF00009FE
:1039300001E0FBD700EBE6FF3FEC4BF041E901EB88
:10394000E6FF02EBE6FFA4EC4AF042E941E9E7CFEB
:10395000D9FF1200D9CFE6FFE1CFD9FF83E9E7EC29
:103960004BF0000901E0FBD700EBE6FF3FEC4BF02A
:1039700041E9E7EC4BF0000901E0FBD701EBE6FF82
:10398000B9EC4BF041E941E9E7CFD9FF1200D9CFBB
:10399000E6FFE1CFD9FF82E9E7EC4BF0000901E057
:1039A000FBD700EBE6FF3FEC4BF041E941E9E7CF05
:1039B000D9FF1200D9CFE6FFE1CFD9FF81E941E875
:1039C000E7EC4BF0000901E0FBD7080EE66E58EC7F
:1039D0004BF041E9016A080E015C13E2E7EC4BF0A1
:1039E000000901E0FBD70150F76AD80FF66E980E78
:1039F000F7220800F5CFE6FFB9EC4BF041E9012AC8
:103A0000EAD742E9E7CFD9FF1200D9CFE6FFE1CFED
:103A1000D9FF85E90A0EE66EE66A00EBE6FF01EBE8
:103A2000E6FFD0EC32F042E9F3CFE6FFF4CFE6FF59
:103A3000A0EC3BF00A0EE66EE66A00EBE6FF01EB57
:103A4000E6FF9DEC3BF01E0EE66E670EE66EE66A44
:103A500002EBE6FF03EBE6FF80EC49F049E90A0ED2
:103A6000E66EE66A00EBE6FF01EBE6FF9DEC3BF05D
:103A7000E552E5CFDCF0E7CFDBF00001DB51DC11F4
:103A800009E1013407E30228E96E000E0320EA6E23
:103A90002D0EEF6E41E9E7CFD9FF1200010EE66E61
:103AA00053EC4CF041E90000000000000000000071
:103AB00000000000000012003C0EE66E0CEC4CF022
:103AC00041E91200140EE66E0CEC4CF041E91200D4
:103AD000D9CFE6FFE1CFD9FF81E944E800010051E9
:103AE000680A02E115EF28F00F0A02E1B0EF27F0B3
:103AF000010A02E14BEF27F0030A02E1E6EF26F0AC
:103B0000520A02E192EF26F0010A02E11CEF26F0D0
:103B1000030A02E1A8EF25F0010A02E15EEF25F0B9
:103B2000070A02E1F3EF24F0010A02E1A2EF24F018
:103B3000030A02E158EF24F0010A02E10DEF24F03C
:103B40001F0A02E1C2EF23F0010A02E170EF23F045
:103B5000030A02E125EF23F0010A02E1D3EF22F08C
:103B6000070A02E17EEF22F0010A02E130EF22F0C3
:103B7000030A02E1DDEF21F04D0A01E1CDD34C0A49
:103B800001E1F7D2700A01E1A4D2090A01E136D2BB
:103B9000030A01E133D2010A01E130D2070A01E14F
:103BA0002DD2010A01E12AD2030A01E127D2010A3A
:103BB00001E124D2070A01E1D1D1470A01E189D10B
:103BC000010A01E144D1030A01E1EFD0010A01E158
:103BD00078D01E0A50E0010A4EE0070A4CE0030AC2
:103BE0004AE00F0A06E0010A04E0030A02E07AEF65
:103BF00028F0000147511DE0000E0001E76E471953
:103C000002E7473502D04751E75C07E2020E0001A8
:103C1000005D03E20001002B09D00001473506E3F7
:103C200000010051000802E2000100070001476B9B
:103C300020D081B41ED0026A036A046A8150040B4A
:103C400012E1400E025C0D0E0358030E04580BE205
:103C5000D950020FE96EDACFEAFFEE2A000EEE220B
:103C6000000EEE22EBD70001140E006F0001150EBE
:103C7000026F7BEF28F00001475103E00001476B22
:103C80001ED081B41CD0026A036A046A8150040BFE
:103C900012E1400E025C0D0E0358030E04580BE2B5
:103CA000D950020FE96EDACFEAFFEE2A000EEE22BB
:103CB000000EEE22EBD70001006B0001026B7BEFE0
:103CC00028F0000147511DE0000E0001E76E471982
:103CD00002E7473502D04751E75C07E21A0E0001C0
:103CE000025D03E20001022B09D00001473506E323
:103CF00000010251140802E2000102070001476BB3
:103D000052D081B450D0026A036A046A8150040B15
:103D100012E1400E025C0D0E0358030E04580BE234
:103D2000D950020FE96EDACFEAFFEE2A000EEE223A
:103D3000000EEE22EBD7000102511A0A29E0020A16
:103D400020E00F0A18E0010A10E0030A06E0010A69
:103D500001E028D00001006B26D00001150E006F95
:103D600008C004F009C005F01ED00001160E006F57
:103D700006C002F018D00001170E006F48C002F014
:103D800012D00001280E006F0001290E026F0BD027
:103D90000001065106E10001500E006F0001510EB6
:103DA000026F01D000D07BEF28F0000147512BE0DB
:103DB00047C0DBF00001DC6BDBBFDC690001DB51DD
:103DC000000104270001DC51000105230001476BBD
:103DD000960E0001D89005BF03D0045D000E055972
:103DE00005E2960E0001046F056B0CD0000105354D
:103DF00004E20451FA08000E055504E2FA0E00012F
:103E0000046F056B22D081B420D0026A036A046A71
:103E10008150040B12E1400E025C0D0E0358030E9C
:103E200004580BE2D950020FE96EDACFEAFFEE2A0E
:103E3000000EEE22000EEE22EBD704C008F005C003
:103E400009F030EC3EF00001006B7BEF28F0000140
:103E500047511DE0000E0001E76E471902E74735A4
:103E600002D04751E75C07E2020E0001025D03E267
:103E70000001022B09D00001473506E30001025181
:103E8000000802E2000102070001476B20D081B464
:103E90001ED0026A036A046A8150040B12E1400ECC
:103EA000025C0D0E0358030E04580BE2D950020FAA
:103EB000E96EDACFEAFFEE2A000EEE22000EEE22C5
:103EC000EBD702C006F030EC3EF00001006B7BEF58
:103ED00028F0000147511DE0000E0001E76E471970
:103EE00002E7473502D04751E75C07E2020E0001C6
:103EF000025D03E20001022B09D00001473506E311
:103F000000010251010802E2000102070001476BB3
:103F100023D081B421D0026A036A046A8150040B61
:103F200012E1400E025C0D0E0358030E04580BE222
:103F3000D950020FE96EDACFEAFFEE2A000EEE2228
:103F4000000EEE22EBD702C048F030EC3EF000014C
:103F5000640E496F0001006B7BEF28F000014751B0
:103F60001DE0000E0001E76E471902E7473502D059
:103F70004751E75C07E2580E0001025D03E20001D1
:103F8000022B09D00001473506E300010251500819
:103F900002E2000102070001476B2ED081B42CD051
:103FA000026A036A046A8150040B12E1400E025C4B
:103FB0000D0E0358030E04580BE2D950020FE96EA0
:103FC000DACFEAFFEE2A000EEE22000EEE22EBD749
:103FD000500E0001025D0BE10001006B8D92899E85
:103FE000899C8B908B928B948B968B9802D002C07D
:103FF00000F00001010E026F7BEF28F00001475135
:1040000047E0000E0001E76E471902E7473502D08E
:104010004751E75C02E2016A05D00001473502E33F
:10402000010E016E0001476B00010051570A29E0A3
:10403000010A21E0030A19E0010A11E0070A09E078
:10404000010A01E024D00150E8B08D82E8A08D92F1
:104050001FD00150E8B08B86E8A08B9619D0015094
:10406000E8B08B88E8A08B9813D00150E8B08B841F
:10407000E8A08B940DD00150E8B08B82E8A08B9221
:1040800007D00150E8B08B80E8A08B9001D000D021
:1040900081B41DD0026A036A046A8150040B12E1E4
:1040A000400E025C0D0E0358030E04580BE2D9506B
:1040B000020FE96EDACFEAFFEE2A000EEE22000EC2
:1040C000EE22EBD700C002F00001500E006F7BEF34
:1040D00028F0000147512BE0000E0001E76E471960
:1040E00002E7473502D04751E75C07E2020E0001C4
:1040F000025D03E20001022B09D00001473506E30F
:1041000000010251000802E2000102070001476BB2
:104110000001025103E1899E898C09D0020E000141
:10412000025D03E1899C898E02D0899C899E81B4BD
:104130001ED0026A036A046A8150040B12E1400E29
:10414000025C0D0E0358030E04580BE2D950020F07
:10415000E96EDACFEAFFEE2A000EEE22000EEE2222
:10416000EBD70001580E026F0001500E006F7BEF7D
:1041700028F0000147511DE0000E0001E76E4719CD
:1041800002E7473502D04751E75C07E2370E0001EE
:10419000025D03E20001022B09D00001473506E36E
:1041A00000010251280802E2000102070001476BEA
:1041B000B1D081B4AFD0026A036A046A8150040BA3
:1041C00012E1400E025C0D0E0358030E04580BE280
:1041D000D950020FE96EDACFEAFFEE2A000EEE2286
:1041E000000EEE22EBD7400E025C0D0E0358030EBC
:1041F000045809E30001640E006F0001650E026FB0
:104200008AEC3EF087D0280E0001025D05E1000136
:10421000006B8AEC3EF07ED002C000F0000102513B
:10422000370A72E0010A6BE0030A64E0010A5CE00D
:10423000070A53E0010A4AE0030A42E0010A39E0B2
:104240001F0A30E0010A27E0030A1EE0010A16E017
:10425000070A0FE0010A08E0030A01E05AD00AC089
:1042600004F00BC005F056D00CC004F00DC005F0F2
:1042700051D00EC004F00FC005F04CD000011E510B
:104280000001046F056B46D010C004F00001056BFF
:1042900004BF05693FD011C004F00001056B04BFE5
:1042A000056938D012C004F00001056B04BF056930
:1042B00031D013C004F00001056B04BF05692AD09A
:1042C000000114510001046F056B24D015C004F0E7
:1042D0000001056B04BF05691DD016C004F0000184
:1042E000056B04BF056916D0000117510001046F6A
:1042F000056B10D018C004F019C005F00BD01AC01F
:1043000004F01BC005F006D01CC004F01DC005F071
:1043100001D000D07BEF28F0000147511DE0000ED6
:104320000001E76E471902E7473502D04751E75CC5
:1043300007E2680E0001025D03E20001022B09D0D2
:104340000001473506E300010251640802E2000162
:1043500002070001476B2FD081B42DD081A4FED776
:10436000640E0001025D05E10001006B8AEC3EF085
:1043700022D002C000F000010251680A16E00F0AC4
:104380000FE0010A08E0030A01E014D023C004F0A2
:1043900024C005F010D029C004F02AC005F00BD0CD
:1043A0002FC004F030C005F006D035C004F036C090
:1043B00005F001D000D07BEF28F0000147512AE042
:1043C00047C0DBF00001DC6BDBBFDC690001DB51C7
:1043D000000104270001DC51000105230001476BA7
:1043E0000001D880055104E7EC0E045DFF0E05596D
:1043F00005E20001EC0E046F05690BD000010535E4
:1044000004E204510008000E055503E20001046BAC
:10441000056B24D081B422D0026A036A046A8150F9
:10442000040B12E1400E025C0D0E0358030E0458FB
:104430000BE2D950020FE96EDACFEAFFEE2A000E46
:10444000EE22000EEE22EBD704C00AF005C00BF0FE
:104450000001280E006F0001290E026F7BEF28F08B
:104460000001475125E047C0DBF00001DC6BDBBFFA
:10447000DC690001DB51000104270001DC5100016F
:1044800005230001476B0001053504E30001046BBF
:10449000056B0DD00001053504E20451C208010E80
:1044A000055505E20001C20E046F010E056F24D010
:1044B00081B422D0026A036A046A8150040B12E1BB
:1044C000400E025C0D0E0358030E04580BE2D95047
:1044D000020FE96EDACFEAFFEE2A000EEE22000E9E
:1044E000EE22EBD704C00CF005C00DF00001280E41
:1044F000006F00012A0E026F7BEF28F00001475188
:104500002CE047C0DBF00001DC6BDBBFDC690001A5
:10451000DB51000104270001DC51000105230001EB
:10452000476BFA0E0001D89005BF03D0045D000E62
:10453000055905E2FA0E0001046F056B0DD000016C
:10454000053504E204515808020E055505E2000144
:10455000580E046F020E056F24D081B422D0026A77
:10456000036A046A8150040B12E1400E025C0D0ED6
:104570000358030E04580BE2D950020FE96EDACF4C
:10458000EAFFEE2A000EEE22000EEE22EBD704C068
:104590000EF005C00FF00001280E006F00012B0E79
:1045A000026F7BEF28F0000147512BE047C0DBF0A2
:1045B0000001DC6BDBBFDC690001DB51000104277B
:1045C0000001DC51000105230001476B320E0001A0
:1045D000D89005BF03D0045D000E055905E2320EE8
:1045E0000001046F056B0CD00001053504E2045195
:1045F000C808000E055504E2C80E0001046F056BE3
:1046000022D081B420D0026A036A046A8150040B6C
:1046100012E1400E025C0D0E0358030E04580BE22B
:10462000D950020FE96EDACFEAFFEE2A000EEE2231
:10463000000EEE22EBD704C01EF00001280E006F22
:1046400000012C0E026F7BEF28F00001475124E09F
:1046500047C0DBF00001DC6BDBBFDC690001DB5134
:10466000000104270001DC51000105230001476B14
:104670000001053504E30001046B056B0CD000015B
:10468000053504E20451C808000E055504E2C80EC1
:104690000001046F056B22D081B420D0026A036A46
:1046A000046A8150040B12E1400E025C0D0E0358A7
:1046B000030E04580BE2D950020FE96EDACFEAFF7D
:1046C000EE2A000EEE22000EEE22EBD704C010F010
:1046D0000001280E006F00012D0E026F7BEF28F005
:1046E000000147512BE047C0DBF00001DC6BDBBF72
:1046F000DC690001DB51000104270001DC510001ED
:1047000005230001476B0001D880055104E79C0E8A
:10471000045DFF0E055905E200019C0E046F05695A
:104720000CD00001053504E204516408000E055563
:1047300004E2640E0001046F056B22D081B420D026
:10474000026A036A046A8150040B12E1400E025CA3
:104750000D0E0358030E04580BE2D950020FE96EF8
:10476000DACFEAFFEE2A000EEE22000EEE22EBD7A1
:1047700004C011F00001280E006F00012E0E026F20
:104780007BEF28F00001475124E047C0DBF0000137
:10479000DC6BDBBFDC690001DB5100010427000199
:1047A000DC51000105230001476B0001053504E3DE
:1047B0000001046B056B0CD00001053504E20451C7
:1047C0001E08000E055504E21E0E0001046F056B65
:1047D00022D081B420D0026A036A046A8150040B9B
:1047E00012E1400E025C0D0E0358030E04580BE25A
:1047F000D950020FE96EDACFEAFFEE2A000EEE2260
:10480000000EEE22EBD704C012F00001280E006F5C
:1048100000012F0E026F7BEF28F00001475124E0CA
:1048200047C0DBF00001DC6BDBBFDC690001DB5162
:10483000000104270001DC51000105230001476B42
:104840000001053504E30001046B056B0CD0000189
:10485000053504E204513C08000E055504E23C0E07
:104860000001046F056B22D081B420D0026A036A74
:10487000046A8150040B12E1400E025C0D0E0358D5
:10488000030E04580BE2D950020FE96EDACFEAFFAB
:10489000EE2A000EEE22000EEE22EBD704C013F03B
:1048A0000001280E006F0001300E026F7BEF28F030
:1048B0000001475124E047C0DBF00001DC6BDBBFA7
:1048C000DC690001DB51000104270001DC5100011B
:1048D00005230001476B0001053504E30001046B6B
:1048E000056B0CD00001053504E204513208000EBE
:1048F000055504E2320E0001046F056B22D081B42D
:1049000020D0026A036A046A8150040B12E1400E4F
:10491000025C0D0E0358030E04580BE2D950020F2F
:10492000E96EDACFEAFFEE2A000EEE22000EEE224A
:10493000EBD704C014F00001280E006F0001310E07
:10494000026FD9D3000147512BE047C0DBF00001D3
:10495000DC6BDBBFDC690001DB51000104270001D7
:10496000DC51000105230001476B050E0001D890C2
:1049700005BF03D0045D000E055905E2050E0001D8
:10498000046F056B0CD00001053504E204511408D6
:10499000000E055504E2140E0001046F056B22D0D1
:1049A00081B420D0026A036A046A8150040B12E1C8
:1049B000400E025C0D0E0358030E04580BE2D95052
:1049C000020FE96EDACFEAFFEE2A000EEE22000EA9
:1049D000EE22EBD704C015F00001280E006F000195
:1049E000320E026F88D30001475145E047C0DBF02B
:1049F0000001DC6BDBBFDC690001DB510001042737
:104A00000001DC51000105230001476B0001053561
:104A100004E30001046B056B0CD00001053504E2D2
:104A200004512808000E055504E2280E0001046F09
:104A3000056B020E0001155D0001DB6FDC6B800B66
:104A400001E0DC690001DC35DC510001051908E6F4
:104A50000001DB510001045D0001DC51000105593A
:104A600009E3020E0001155D0001046F056B800B68
:104A700001E0056922D081B420D0026A036A046A89
:104A80008150040B12E1400E025C0D0E0358030E20
:104A900004580BE2D950020FE96EDACFEAFFEE2A92
:104AA000000EEE22000EEE22EBD704C016F000013D
:104AB000280E006F0001330E026F1DD30001475115
:104AC00024E047C0DBF00001DC6BDBBFDC690001E8
:104AD000DB51000104270001DC5100010523000126
:104AE000476B0001053504E30001046B056B0CD036
:104AF0000001053504E204510208000E055504E2E8
:104B0000020E0001046F056B22D081B420D0026A2E
:104B1000036A046A8150040B12E1400E025C0D0E20
:104B20000358030E04580BE2D950020FE96EDACF96
:104B3000EAFFEE2A000EEE22000EEE22EBD704C0B2
:104B400017F00001280E006F0001340E026FD3D25F
:104B5000000147514CE047C0DBF00001DC6BDBBFDC
:104B6000DC690001DB51000104270001DC51000178
:104B700005230001476B0001D880055104E7380E7A
:104B8000045DFF0E055905E20001380E046F05694A
:104B90000CD00001053504E20451C808000E05558B
:104BA00004E2C80E0001046F056B1AC0DBF01BC0E5
:104BB000DCF000010A0EDB5F000EDC5B0001053556
:104BC00005510001DC1908E6000104510001DB5D1C
:104BD000000105510001DC5909E21AC004F01BC0B4
:104BE00005F000010A0E045F000E055B24D081B4BD
:104BF00022D0026A036A046A8150040B12E1400E5B
:104C0000025C0D0E0358030E04580BE2D950020F3C
:104C1000E96EDACFEAFFEE2A000EEE22000EEE2257
:104C2000EBD704C018F005C019F00001280E006F82
:104C30000001350E026F5FD2000147514EE047C0C0
:104C4000DBF00001DC6BDBBFDC690001DB51000144
:104C500004270001DC51000105230001476B00011E
:104C6000D880055104E7380E045DFF0E055905E2B2
:104C70000001380E046F05690CD00001053504E20F
:104C80000451C808000E055504E2C80E0001046F67
:104C9000056B0A0E000118250001DB6F000E0001F4
:104CA00019210001DC6F0001DC35DC510001051920
:104CB00008E60001DB510001045D0001DC51000148
:104CC00005590AE20A0E000118250001046F000EC2
:104CD000000119210001056F24D081B422D0026A9D
:104CE000036A046A8150040B12E1400E025C0D0E4F
:104CF0000358030E04580BE2D950020FE96EDACFC5
:104D0000EAFFEE2A000EEE22000EEE22EBD704C0E0
:104D10001AF005C01BF00001280E006F0001360ECE
:104D2000026FE9D1000147512CE047C0DBF00001E0
:104D3000DC6BDBBFDC690001DB51000104270001F3
:104D4000DC51000105230001476B640E0001D8907F
:104D500005BF03D0045D000E055905E2640E000195
:104D6000046F056B0DD00001053504E20451F40811
:104D7000010E055505E20001F40E046F010E056FEA
:104D800024D081B422D0026A036A046A8150040BE1
:104D900012E1400E025C0D0E0358030E04580BE2A4
:104DA000D950020FE96EDACFEAFFEE2A000EEE22AA
:104DB000000EEE22EBD704C01CF005C01DF0000170
:104DC000280E006F0001370E026F95D10001475188
:104DD0003DE047C0DBF00001DC6BDBBFDC690001BC
:104DE000DB51000104270001DC5100010523000113
:104DF000476B700E0001231902E1170E241921E000
:104E0000880E0001231902E1130E24191AE0000193
:104E1000D880055104E7CE0E045DFF0E055905E26A
:104E20000001CE0E046F05690CD00001053504E2C7
:104E300004513208000E055504E2320E0001046FE1
:104E4000056B04C023F005C024F024D081B422D027
:104E5000026A036A046A8150040B12E1400E025C8C
:104E60000D0E0358030E04580BE2D950020FE96EE1
:104E7000DACFEAFFEE2A000EEE22000EEE22EBD78A
:104E800004C023F005C024F00001640E006F00018F
:104E9000650E026F30D1000147513DE047C0DBF0A5
:104EA0000001DC6BDBBFDC690001DB510001042782
:104EB0000001DC51000105230001476B700E000169
:104EC000291902E1170E2A1921E0880E000129197B
:104ED00002E1130E2A191AE00001D880055104E7F7
:104EE000CE0E045DFF0E055905E20001CE0E046FE3
:104EF00005690CD00001053504E204513208000EAA
:104F0000055504E2320E0001046F056B04C029F060
:104F100005C02AF024D081B422D0026A036A046A50
:104F20008150040B12E1400E025C0D0E0358030E7B
:104F300004580BE2D950020FE96EDACFEAFFEE2AED
:104F4000000EEE22000EEE22EBD704C029F005C0C1
:104F50002AF00001640E006F0001660E026FCBD0D4
:104F6000000147513DE047C0DBF00001DC6BDBBFD7
:104F7000DC690001DB51000104270001DC51000164
:104F800005230001476B700E00012B1902E1170E7B
:104F90002C1921E0880E00012B1902E1130E2C19A7
:104FA0001AE00001D880055104E7CE0E045DFF0E23
:104FB000055905E20001CE0E046F05690CD0000111
:104FC000053504E204513208000E055504E2320EA4
:104FD0000001046F056B04C02FF005C030F024D031
:104FE00081B422D0026A036A046A8150040B12E180
:104FF000400E025C0D0E0358030E04580BE2D9500C
:10500000020FE96EDACFEAFFEE2A000EEE22000E62
:10501000EE22EBD704C02FF005C030F00001640E83
:10502000006F0001670E026F66D0000147513DE03E
:1050300047C0DBF00001DC6BDBBFDC690001DB514A
:10504000000104270001DC51000105230001476B2A
:10505000700E0001351902E1170E361921E0880E95
:105060000001351902E1130E36191AE00001D8804B
:10507000055104E7CE0E045DFF0E055905E200015F
:10508000CE0E046F05690CD00001053504E2045111
:105090003208000E055504E2320E0001046F056B64
:1050A00004C035F005C036F024D081B422D0026AA5
:1050B000036A046A8150040B12E1400E025C0D0E7B
:1050C0000358030E04580BE2D950020FE96EDACFF1
:1050D000EAFFEE2A000EEE22000EEE22EBD704C00D
:1050E00035F005C036F00001640E006F0001680E57
:1050F000026F01D000D045E9E7CFD9FF1200020EC0
:105100000001485D26E10001495121E100013851CB
:1051100003E0000137510AE10001065107E00001F8
:10512000030502E18B8A01D08B9A10D00A0E000190
:10513000005D0BE3000100510F0807E300010305C8
:1051400002E18B8A01D08B9A01D08B9A01D08B8A95
:105150000AD00001480504E18B8A0001496B03D0A5
:085160008B9A0001496B12005B
:08516800D9CFE6FFE1CFD9FF2A
:1051700081E959E865EC46F06CEC46F08B8A1EEC50
:105180001CF0C80EE66E09EC4BF041E9C80EE66E65
:1051900009EC4BF041E9C80EE66E09EC4BF041E931
:1051A000C80EE66E09EC4BF041E9E8EC46F063EC22
:1051B00040F0000106290001076F82EC2FF071EC2E
:1051C0002EF010D808D931DAC3DB66EC32F068EC87
:1051D0001DF07FEC28F014EC00F0EFD75AE9E7CF90
:1051E000D9FF1200000107510001065D01E1F2D074
:1051F000000106510FE10001010E376F0001010EA1
:10520000386F00013C6B8D928B948B908B928B96B8
:105210008B98DED0000106056BE10001030E006FE4
:1052200014EC00F00001010E376F0001010E386F21
:105230008D92C80EE66E09EC4BF041E9C80EE66EA1
:1052400009EC4BF041E98B96C80EE66E09EC4BF089
:1052500041E9C80EE66E09EC4BF041E9C80EE66E76
:1052600009EC4BF041E9C80EE66E09EC4BF041E960
:10527000C80EE66E09EC4BF041E9C80EE66E09EC8B
:105280004BF041E98B98C80EE66E09EC4BF041E912
:10529000C80EE66E09EC4BF041E9C80EE66E09EC6B
:1052A0004BF041E9C80EE66E09EC4BF041E9C80E3F
:1052B000E66E09EC4BF041E98B848D82899C899ED6
:1052C00000013D6B00013E6B00013F6B406B000134
:1052D000416B426B0001436B446B640E0001456FF0
:1052E000466B0001010E3C6F8B880001006B70D093
:1052F000020E0001065D6CE10001040E006F14EC6B
:1053000000F00001010E376F0001010E386F8D9221
:10531000C80EE66E09EC4BF041E9C80EE66E09ECEA
:105320004BF041E98B86C80EE66E09EC4BF041E983
:10533000C80EE66E09EC4BF041E9C80EE66E09ECCA
:105340004BF041E9C80EE66E09EC4BF041E9C80E9E
:10535000E66E09EC4BF041E9C80EE66E09EC4BF045
:1053600041E98B88C80EE66E09EC4BF041E9C80EA6
:10537000E66E09EC4BF041E9C80EE66E09EC4BF025
:1053800041E9C80EE66E09EC4BF041E9C80EE66E45
:1053900009EC4BF041E98B928B848D82899C899E2C
:1053A00000013D6B00013E6B00013F6B406B000153
:1053B000416B426B0001436B446B640E0001456F0F
:1053C000466B0001010E3C6F8B980001006B00D012
:1053D00006C007F01200D9CFE6FFE1CFD9FF81E97F
:1053E00042E88450040B33E10001390530E1016AE1
:1053F000026A8450040B16E101EBDBF002EBDCF0F7
:105400000001DD6B0001D890DD51000A06E6500E68
:10541000DB5DC30EDC59000EDD5904E2012A000EEB
:105420000222E7D701EBDBF002EBDCF00001DD6BE1
:105430000001D890DD51000A06E6500EDB5DC30E78
:10544000DC59000EDD5902E30001396B36D084507F
:10545000040B33E00001395130E1016A026A8450E3
:10546000040B16E001EBDBF002EBDCF00001DD6B7E
:105470000001D890DD51000A06E6500EDB5DC30E38
:10548000DC59000EDD5904E2012A000E0222E7D7A2
:1054900001EBDBF002EBDCF00001DD6B0001D890EA
:1054A000DD51000A06E6500EDB5DC30EDC59000E2E
:1054B000DD5903E30001010E396F000106055BE1D0
:1054C00015C0DDF00001DE6BDDBFDE69000100010B
:1054D00008510001DD250001DB6F000100010951C9
:1054E0000001DE210001DC6F0001DC35DC51000130
:1054F000221908E60001DB510001215D0001DC51A9
:105500000001225904E300013C6B8B942AD016C0A1
:10551000DDF00001DE6BDDBFDE6900010001085136
:105520000001DD250001DB6F0001000109510001D0
:10553000DE210001DC6F0001223522510001DC195F
:1055400008E6000121510001DB5D0001225100014C
:10555000DC5907E300013C5104E10001010E3C6FFE
:105560008B840001375106E100013C0503E1000195
:10557000030E3C6F10D0020E0001065D0AE100012F
:10558000370505E10001010E3C6F8B8401D08B943F
:1055900002D000013C6B500E0001005D42E20001B0
:1055A00017050AE10001060507E18B50040B02E034
:1055B0008B8001D08B9035D0020E0001175D30E159
:1055C000000106052DE18B50040B11E0000134357C
:1055D00034510001191908E6000133510001185D2A
:1055E000000134510001195902E38B8018D08B500F
:1055F000040B11E000011B351B510001341908E6B2
:1056000000011A510001335D00011B5100013459A2
:1056100002E38B9004D08BB402D08B9000D001D0E9
:105620008B9043E9E7CFD9FF1200D9CFE6FFE1CF56
:10563000D9FF81E942E88450010B32E10001375182
:105640002FE0016A026A8450010B16E101EBDBF0E6
:1056500002EBDCF00001DD6B0001D890DD51000AA7
:1056600006E6500EDB5DC30EDC59000EDD5904E288
:10567000012A000E0222E7D701EBDBF002EBDCF09F
:105680000001DD6B0001D890DD51000A06E6500EE6
:10569000DB5DC30EDC59000EDD5902E30001376B00
:1056A0000001060501E0F7D0000137514FE18B887A
:1056B00000010F350F510001281908E600010E51B5
:1056C0000001275D00010F510001285903E200018C
:1056D0003C5102E18B9239D00A0E00013A250001BB
:1056E000DB6F000E00013B210001DC6F0001DC35A7
:1056F000DC5100012E1908E60001DB5100012D5D8F
:105700000001DC5100012E5902E38B921ED03AC0F9
:10571000DBF03BC0DCF000010A0EDB5F000EDC5B5F
:1057200000012E352E510001DC1908E600012D5133
:105730000001DB5D00012E510001DC5906E3030E80
:1057400000013C5D01E18B8200D0A4D000010F3547
:105750000F510001281908E600010E510001275DD4
:1057600000010F510001285903E38B888B9241D02F
:1057700010C0DDF00001DE6BDDBFDE69000100015D
:105780003A510001DD250001DB6F000100013B51B2
:105790000001DE210001DC6F0001283528510001E5
:1057A000DC1908E6000127510001DB5D00012851EA
:1057B0000001DC5906E300013C0502E18B9800D0B2
:1057C00018D08B50010B15E000012835285100013D
:1057D0001D1908E60001275100011C5D0001285138
:1057E00000011D5906E300013C0502E18B9800D041
:1057F00000D08B50100B31E111C0DBF00001DC6BED
:10580000DBBFDC690001343534510001DC1908E6E6
:10581000000133510001DB5D000134510001DC590E
:105820001CE33AC0DBF03BC0DCF00001140EDB5F90
:10583000000EDC5B00012E352E510001DC1908E65C
:1058400000012D510001DB5D00012E510001DC59EA
:1058500004E300013C0501E18B828B50020B1AE04E
:10586000640E00013A250001DB6F000E00013B21B0
:105870000001DC6F0001DC35DC510001281908E66D
:105880000001DB510001275D0001DC5100012859B6
:1058900001E38B9259D0020E0001065D4BE100013D
:1058A000375102E18B9845D00001283504E2275199
:1058B0003208000E285514E200011E510001DB6F72
:1058C000DC6B0001283528510001DC1908E60001D5
:1058D00027510001DB5D000128510001DC5902E382
:1058E0008B9827D010C0DDF00001DE6BDDBFDE69D4
:1058F0000001DD5100013A5D0001DB6F0001DE5166
:1059000000013B590001DC6F0001DC35DC51000176
:10591000281908E60001DB510001275D0001DC5178
:105920000001285906E300013C0502E18B8800D004
:1059300000D00AD0500E0001005D06E28D928B94DB
:105940008B908B928B968B9843E9E7CFD9FF12000F
:10595000D9CFE6FFE1CFD9FF81E942E80001065146
:1059600001E18CD100013C5102E194D986D1030EB2
:1059700000013C5D02E1A1D980D100013C0501E0BC
:105980007CD100012D5100013A5D016E3B510001B7
:105990002E55026E01EBE6FF02EBE6FFD0EC32F093
:1059A00042E9F3CFDBF0F4CFDCF00001DC3504E2B8
:1059B000DB511408000EDC5505E20A0E0001456FAC
:1059C000466B34D001EBE6FF02EBE6FFD0EC32F0A1
:1059D00042E9F3CFDBF0F4CFDCF00001DC3504E288
:1059E000DB510A08000EDC5505E2140E0001456F7C
:1059F000466B1CD001EBE6FF02EBE6FFD0EC32F089
:105A000042E9F3CFDBF0F4CFDCF00001DC3504E257
:105A1000DB510508000EDC5505E21E0E0001456F46
:105A2000466B04D0640E0001456F466B01EBE6FF48
:105A300002EBE6FFD0EC32F042E9F3CFDBF0F4CF3B
:105A4000DCF0020E0001D890DCBF03D0DB5D000E5D
:105A5000DC5903E30001010E3E6F0150021007E123
:105A6000899C899E00013D6B0001416B426B0001E6
:105A7000455100013F5D000146510001405975E369
:105A800000013E0572E100013F6B406B01EBE6FF58
:105A900002EBE6FFD0EC32F042E9F3CFDBF0F4CFDB
:105AA000DCF00001DC3504E2DB510A08000EDC55B5
:105AB00010E201EB41F002EB42F00001030E420361
:105AC000F3CF42F0030E4103F3CF41F0F4504227ED
:105AD0004CD001EBE6FF02EBE6FFD0EC32F042E9FE
:105AE000F3CFDBF0F4CFDCF00001DC3504E2DB5176
:105AF0000508000EDC550CE201EB41F002EB42F030
:105B00000001D89041374237D890413742372DD0E5
:105B100001EBE6FF02EBE6FFD0EC32F042E9F3CF17
:105B2000DBF0F4CFDCF0020E0001D890DCBF03D034
:105B3000DB5D000EDC5910E301EB41F002EB42F0BB
:105B40000001070E4203F3CF42F0070E4103F3CFEB
:105B500041F0F450422709D000013D5106E1000117
:105B60003E6B640E00013F6F406B0001423504E262
:105B700041510008000E42553CE241C0E6FF42C0E0
:105B8000E6FFD0EC32F042E9F3CFDBF0F4CFDCF00B
:105B90000001DB5100013F5D0001DC510001405973
:105BA00019E20001D890445104E6A40E435D060EAC
:105BB000445910E2020E0001065D06E1899C898EBF
:105BC0000001030E3D6F05D0898C899E0001020EF5
:105BD0003D6F07D0899C899E00013D6B0001416BA0
:105BE000426B0001443504E341C043F042C044F03D
:105BF00043D00001423540E341C0E6FF42C0E6FF2A
:105C0000D0EC32F042E9F3CFDBF0F4CFDCF000016E
:105C1000DB5100013F5D0001DC510001405918E2F9
:105C20000001443504E343515C08F90E445510E289
:105C3000020E0001065D06E1898C899E0001020EBC
:105C40003D6F05D0899C898E0001030E3D6F07D002
:105C5000899C899E00013D6B0001416B426B0001F4
:105C6000443504E243510008000E445504E241C0AB
:105C700043F042C044F000D000D008D0500E0001E4
:105C8000005D04E2899C899E00013D6B43E9E7CFFA
:105C9000D9FF12000001443504E343515C08F90EBA
:105CA000445506E2899C898E0001030E3D6F04D0A5
:105CB000899C899E00013D6B12000001D8904451DF
:105CC00004E6A40E435D060E445906E2898C899EC3
:105CD0000001020E3D6F04D0899C899E00013D6B3E
:105CE0001200D9CFE6FFE1CFD9FF81E949E80001F1
:105CF000060501E0DBD00001395104E10001145137
:105D0000096E01D0096A13C0DDF00001DE6BDDBF52
:105D1000DE69DDC0E6FFDEC0E6FF000121510001C3
:105D2000085D0001DB6F00012251000109590001EB
:105D3000DC6FDBC0E6FFDCC0E6FFA6EC3CF0E55222
:105D4000E550086EE750076E0A0EE66EE66A07EB4E
:105D5000E6FF08EBE6FF9DEC3BF0E552E550086EF0
:105D6000E750076E083404E207501408000E085488
:105D700004E2140E076E086A0BD0D880085004E7BE
:105D8000EC0E075CFF0E085803E2EC0E076E086885
:105D900009EBE6FF10EC3BF007EBE6FF08EBE6FF54
:105DA0002FEC3BF0E66AE66A200EE66E410EE66EE8
:105DB00012C0E6FF12EC3BF0E66AE66A480EE66EB9
:105DC000430EE66E08C0E6FF09C0E6FF2FEC3BF08D
:105DD000E0EC39F0DAEC3CF0D9EC3BF00CC0E6FF3B
:105DE0000DC0E6FF2FEC3BF0E66AE66A200EE66E99
:105DF000410EE66E0AC0E6FF0BC0E6FF2FEC3BF05B
:105E000033C0E6FF34C0E6FF2FEC3BF0DAEC3CF0A9
:105E1000D9EC3BF0E2EC39F0E2EC39F0E2EC39F0AD
:105E2000E2EC39F0E552E5CFDEF0E5CFDDF0E5CF8D
:105E3000DCF0E7CFDBF00001DB51016EDC51026EDC
:105E4000DD51036EDE51046E01EBE6FF02EBE6FF6F
:105E500003EBE6FF04EBE6FFC2DB44E900013A5145
:105E6000F35C056E3B51F458066E05EBE6FF06EB5E
:105E7000E6FF96DB42E9F3CFDBF0F4CFDCF0000184
:105E8000DC3504E2DB510208000EDC550EE201EBCA
:105E9000E6FF02EBE6FF03EBE6FF04EBE6FF9FDB2A
:105EA00044E9F3CF3AF0F4CF3BF00DD0020E0001FD
:105EB000065D05E108C03AF009C03BF004D008C017
:105EC0003AF009C03BF000013B3504E23A51C20808
:105ED000010E3B5506E20001C20E3A6F010E3B6F08
:105EE0000DD0960E0001D8903BBF03D03A5D000E56
:105EF0003B5904E2960E00013A6F3B6B4AE9E7CF4B
:105F0000D9FF1200D9CFE6FFE1CFD9FF81E946E8FA
:105F10000A0E00014A5D0AE2650E0001005D01E023
:105F20007DD0010E00014A5D01E278D0830EE66E5D
:105F3000D0EC4BF041E9140EE66E0CEC4CF041E96C
:105F400073EC4CF067EC4CF0000901E0FBD7020E5B
:105F5000E66EE66A47EC4CF0F350000123250001A1
:105F6000DD6FF450000124210001DE6F000100010B
:105F70001F510001DD250001DB6F000100012051F0
:105F80000001DE210001DC6FDBC0E6FFDCC0E6FFC4
:105F90009DEC3BF0E552E5CF20F0E7CF1FF01FC0AE
:105FA000E6FF20C0E6FFB2D942E9F3CF21F0F4CFFB
:105FB00022F047EC4CF0F3CFDBF0F4CFDCF0000143
:105FC000DC3504E2DB51A0080F0EDC550BE20001CA
:105FD000386B0001700E1F6F170E206F08C021F084
:105FE00009C022F047EC4CF0F3CFDBF0F4CFDCF04B
:105FF000640E0001D890DCBF03D0DB5D000EDC59DD
:106000000BE20001386B0001880E1F6F130E206F2A
:1060100008C021F009C022F000014A6B050E000102
:106020004B5D08E2660E0001005D74E1010E0001A7
:106030004B5D70E3870EE66ED0EC4BF041E9140E39
:10604000E66E0CEC4CF041E973EC4CF067EC4CF074
:10605000000901E0FBD7020EE66EE66A47EC4CF061
:10606000F350000129250001DD6FF45000012A21C1
:106070000001DE6F0001000125510001DD25000156
:10608000DB6F0001000126510001DE210001DC6F01
:10609000DBC0E6FFDCC0E6FF9DEC3BF0E552E5CF60
:1060A00026F0E7CF25F025C0E6FF26C0E6FF2ED973
:1060B00042E9F3CF27F0F4CF28F047EC4CF0F3CFD0
:1060C000DBF0F4CFDCF00001DC3504E2DB51A008AA
:1060D0000F0EDC5507E20001386B0001700E256FD2
:1060E000170E266F47EC4CF0F3CFDBF0F4CFDCF06B
:1060F000640E0001D890DCBF03D0DB5D000EDC59DC
:1061000007E20001386B0001880E256F130E266F21
:1061100000014B6B020E00014C5D08E2670E0001AE
:10612000005D74E1010E00014C5D70E38B0EE66EC4
:10613000D0EC4BF041E9140EE66E0CEC4CF041E96A
:1061400073EC4CF067EC4CF0000901E0FBD7020E59
:10615000E66EE66A47EC4CF0F35000012F25000193
:10616000DD6FF450000130210001DE6F00010001FD
:106170002B510001DD250001DB6F000100012C51D6
:106180000001DE210001DC6FDBC0E6FFDCC0E6FFC2
:106190009DEC3BF0E552E5CF2CF0E7CF2BF02BC088
:1061A000E6FF2CC0E6FFB2D842E9F3CF2DF0F4CFE2
:1061B0002EF047EC4CF0F3CFDBF0F4CFDCF0000135
:1061C000DC3504E2DB51A0080F0EDC5507E20001CC
:1061D000386B0001700E2B6F170E2C6F47EC4CF0D4
:1061E000F3CFDBF0F4CFDCF0640E0001D890DCBF1D
:1061F00003D0DB5D000EDC5907E20001386B0001C3
:10620000880E2B6F130E2C6F00014C6B0A0E0001D1
:106210004D5D08E2680E0001005D74E1010E0001B1
:106220004D5D70E3930EE66ED0EC4BF041E9140E39
:10623000E66E0CEC4CF041E973EC4CF067EC4CF082
:10624000000901E0FBD7020EE66EE66A47EC4CF06F
:10625000F350000135250001DD6FF45000013621B7
:106260000001DE6F0001000131510001DD25000158
:10627000DB6F0001000132510001DE210001DC6F03
:10628000DBC0E6FFDCC0E6FF9DEC3BF0E552E5CF6E
:1062900032F0E7CF31F031C0E6FF32C0E6FF36D84A
:1062A00042E9F3CF33F0F4CF34F047EC4CF0F3CFC6
:1062B000DBF0F4CFDCF00001DC3504E2DB51A008B8
:1062C0000F0EDC5507E20001386B0001700E316FD4
:1062D000170E326F47EC4CF0F3CFDBF0F4CFDCF06D
:1062E000640E0001D890DCBF03D0DB5D000EDC59EA
:1062F00007E20001386B0001880E316F130E326F18
:1063000000014D6B47E9E7CFD9FF1200D9CFE6FF77
:10631000E1CFD9FF83E94AE8036A046AD89005E32C
:10632000580E076E020E086EC8D0AC0EF66E910EB7
:10633000F76E00500900F55C01500A00F55805E2BF
:10634000D40E076EFE0E086EB8D0600EF66E920E7A
:10635000F76E0900F550005C0A00F550015805E29F
:10636000580E076E020E086EA8D003EBF6FF04EB82
:10637000F7FF010ED890F636F736E806FBE1AC0ED3
:10638000F626910EF7220900F550005C0A00F55040
:10639000015804E2032A000E0422E7D703EBF6FFBC
:1063A00004EBF7FF010ED890F636F736E806FBE16E
:1063B000AC0EF626910EF7220900F5CFE6FF090094
:1063C000F5CFE6FF0304F66E000E0458F76E010EDB
:1063D000D890F636F736E806FBE1AC0EF626910EBD
:1063E000F722FE0EE3500900F55C056E41E9E55029
:1063F0000A00F558066E03EBF6FF04EBF7FF010EFB
:10640000D890F636F736E806FBE1AC0EF626910E8C
:10641000F72200010900F550005CDF6F0A00F5501B
:106420000158E06FDFC0E6FFE0C0E6FF2DEC3BF077
:1064300005EBE6FF06EBE6FF2DEC3BF0E66AE66ACD
:10644000200EE66E410EE66ED9EC3BF0DAEC3CF045
:106450000A0EE66EE66A03EBE6FF04EBE6FFA6EC47
:106460003CF02DEC3BF0E66AE66A960EE66EC30E53
:10647000E66EE2EC39F0E0EC39F0E552E5CFDEF023
:10648000E5CFDDF0E5CFDCF0E7CFDBF00001DB515D
:10649000096EDC510A6EDD510B6EDE510C6E09EB9C
:1064A000E6FF0AEBE6FF0BEBE6FF0CEBE6FF97D807
:1064B00044E9F350076EF450086E07EBF3FF08EB66
:1064C000F4FF00D04BE9E7CFD9FF120000013851AB
:1064D0004CE1000106052AE100012C3504E22B51B4
:1064E0008708130E2C5506E20001066B00010A0E08
:1064F000006F1BD00001323504E231518708130EC2
:10650000325506E20001066B00010B0E006F0DD044
:106510000001263504E225518708130E265505E2B1
:106520000001066B00010C0E006F1FD0020E00016F
:10653000065D1BE100012C3504E22B518708130E88
:106540002C5506E20001066B00010A0E006F0DD00B
:106550000001263504E225518708130E265505E271
:106560000001066B00010C0E006F0001375109E1BC
:10657000020E0001065D05E10001066B00010E0E32
:10658000006F0001D890285104E6580E275D020ED6
:10659000285905E30001066B00010F0E006F120081
:1065A000D9CFE6FFE1CFD9FF83E901340FE300EB58
:1065B000DBF001EBDCF00001DB6DDC1F000EDC2307
:1065C000DBC0F3FFDCC0F4FF06D005D000EBF3FF27
:1065D00001EBF4FF00D041E9E7CFD9FF1200D9CF9A
:1065E000E6FFE1CFD9FF85E942E8E66AE66AE66AB6
:1065F000E66A00EBE6FF01EBE6FF02EBE6FF03EBEA
:10660000E6FF36EC3CF0000941E0E66AE66AE66A3D
:106610003F0EE66E00EBE6FF01EBE6FF02EBE6FF66
:1066200003EBE6FF00EBE6FF01EBE6FF02EBE6FF24
:1066300003EBE6FF4EEC3BF02FEC3BF0E0EC39F0E7
:1066400036EC3CF0000912E100EBE6FF01EBE6FF5F
:1066500002EBE6FF03EBE6FF4EEC3BF0FE0EE3043D
:10666000056E000E41E9E558066E0FD000EBE6FF1F
:1066700001EBE6FF02EBE6FF03EBE6FF4EEC3BF03F
:10668000E552E550066EE750056E40D0E66AE66AD0
:10669000E66A3F0EE66E00EBE6FF01EBE6FF02EB7B
:1066A000E6FF03EBE6FF4EEC3BF02FEC3BF000EB9C
:1066B000E6FF01EBE6FF02EBE6FF03EBE6FFE0ECB3
:1066C00039F036EC3CF0000912E100EBE6FF01EB9B
:1066D000E6FF02EBE6FF03EBE6FF4EEC3BF0FE0EBF
:1066E000E328056E41E9000EE520066E0FD000EBB1
:1066F000E6FF01EBE6FF02EBE6FF03EBE6FF4EEC05
:106700003BF0E552E550066EE750056E05EBF3FFF2
:0E67100006EBF4FF00D043E9E7CFD9FF1200FB
:02671E00253321
:10672000692E253169002020204669726D776172DB
:106730006520205625752E2575202020002020203C
:106740002062792056696E63655F303037202020E3
:10675000200020202045563030372020436F6E74B3
:10676000726F6C20202000436F7272656374696FD2
:106770006E2065787465726965757200436F727218
:10678000656374696F6E2064657061727420504334
:1067900000436F7272656374696F6E20736F6E640D
:1067A00065206561750054656D7065726174757200
:1067B00065203D2025732573200054656E73696F35
:1067C0006E203D202534696D562020002020204376
:1067D0004F5552542D4349524355495420202020AF
:1067E000002020202020534F4E44452020454E209D
:1067F0002020202020002020202020434F4E4E45E6
:106800004354454520202020202000202020202007
:10681000534F4E444520204E4F4E20202020200034
:10682000436F7272656374696F6E2020616D626977
:10683000616E636500202020202065787465726990
:1068400065757265202020202000202020202064F3
:106850006570617274202050432020202020002089
:10686000202020206561752062616C6C6F6E202095
:1068700020202000202020202020616D6269616E90
:106880006365202020202020002020436F72726545
:106890006374696F6E20736F6E6465202000202022
:1068A00020206C6120746F756368652E2E2E202069
:1068B00020200020566575696C6C657A2020726511
:1068C0006C616368657220002D2D2D2043414C4979
:1068D00042524154494F4E20202D2D2D00205B4F18
:1068E00046465D2020204F4E2020204155544F2009
:1068F000200020204F46462020205B4F4E5D202068
:106900004155544F20200020204F46462020202073
:106910004F4E20205B4155544F5D20002020202009
:10692000205B257320205D2020202020200054643F
:106930006570617274205043204020546578743D26
:10694000302573002020202020205B2573205D202F
:10695000202020202020002020206561752020722A
:106960006164696174657572202020002054656D32
:10697000706572617475726520206D696E692E2074
:106980000020636F757075726520207261646961A3
:1069900074657572200061637469766174696F6EE5
:1069A0002072616469617465757200202054656DA0
:1069B0007065726174757265204578742E202000B0
:1069C00020636972637569742020726164696174FF
:1069D00065757220002020204163746976617469B6
:1069E0006F6E202064752020200064652072657021
:1069F00072697365206368617566666167650064C6
:106A00006520636F75707572652063686175666671
:106A1000616765002044656C7461205425732020F3
:106A2000616D6269616E7465200020202068657563
:106A30007265732063726575736573202020002072
:106A40002020537572636861756666652020656EE7
:106A500020202000636F7272656374696F6E20205E
:106A6000616D6269616E636500636F727265637404
:106A7000696F6E2020636F6E7369676E65002020FA
:106A80002020204661637465757220646520202093
:106A90002020006175746F7269736174696F6E2074
:106AA0006170706F696E74002020202054656D70D5
:106AB0006572617475726520202020200020656158
:106AC00075202064656D6172726167652050414375
:106AD00020002044656C7461202074656D706572BF
:106AE00061747572652000636F75707572652050F2
:106AF000414320656E2066726F696400636F757034
:106B00007572652050414320656E2063686175642D
:106B1000002054656D706572617475726520206423
:106B200027656175200020204F6666736574206CB0
:106B30006F6920642765617520200020202047614F
:106B4000696E206C6F6920642765617520202000C4
:106B50002D2D2D2020504152414D4554524553205A
:106B6000202D2D2D00444555582052454C41495368
:106B700020414354494620212000204F50454E20BB
:106B8000205B53544F505D20434C4F534520002011
:106B90004F50454E20202053544F50205B434C4FC4
:106BA00053455D005B4F50454E5D202053544F5080
:106BB0002020434C4F5345200020202020323125F7
:106BC0007320202020205B313725735D202020009A
:106BD0002020205B323125735D202020202031379A
:106BE00025732020202000202020202054257320E1
:106BF0006169722050414320202020200020202065
:106C0000203138257320202020205B323025735D11
:106C1000202020002020205B313825735D2020209B
:106C20002020323025732020202000202020204FDB
:106C30004E2020202020205B4F46465D2020200053
:106C40002020205B4F4E5D2020202020204F4646F4
:106C50002020202000202020636F6D6D616E646510
:106C60002020205041432020200044656661757437
:106C700020504143203D20204143544946200044B8
:106C8000656661757420504143203D20494E414363
:106C90005449460048657572652048432020203DD0
:106CA00020204143544946200048657572652048BC
:106CB000432020203D20494E414354494600205363
:106CC00074617475732064657320656E7472656594
:106CD000732000202020202020332020766F69653B
:106CE000732020202020200020202050696C6F7409
:106CF0006167652076616E6E65202020002020632C
:106D0000697263752E2072616469617465757220A1
:106D100020002020202020206170706F696E742078
:106D2000202020202020002020202063697263750D
:106D30006C617465757220202020200020202020A6
:106D400020542573204149522050414320202020C7
:106D5000200020636F6E7369676E65206427616928
:106D600072205041432000202050696C6F7461678D
:106D7000652020736F7274696520200020202063D5
:106D80006F6D6D616E64652020504143202020208E
:106D900000202050696C6F74616765202072656CFB
:106DA000616973202000202020202020656E7472ED
:106DB0006565732020202020202000202020204CEA
:106DC00065637475726573206465732020202000EC
:106DD0002D204D4F4445204D41494E54454E414E86
:106DE0004345202D005B204F4E205D202020544540
:106DF0004D504F5249534520200020204F4E202017
:106E0000205B2054454D504F52495345205D002092
:106E100020202020204261636B6C69676874202009
:106E2000202020002020202020202045525245559F
:106E30005220202020202020003C20205241465279
:106E400041494348495353454D454E5420003C2049
:106E500020202043484155464641474520202020D8
:106E6000203E002020202020202041525245542046
:106E70002020202020203E004D6F64652020466F9A
:106E80006E6374696F6E6E656D656E740020202090
:106E900020205B25732573205D20202020202000EA
:106EA000436F6E7369676E652054257320416D6270
:106EB00069616E74650020436F6E732E20542573D4
:106EC0002044657061727420504320002D2D2D2DBB
:106ED00020205245474C4147455320202D2D2D2D34
:106EE000002020202020494E54455244495420215E
:106EF00020202020200020204D4F4445204D414996
:106F00004E54454E414E4345202000202020202055
:106F1000456E747265722020656E2020202020004E
:106F20003C2D2D202020202020202020202020202B
:106F300020202020002020202020202020562575E1
:106F40002E2575202020202020202000202056657E
:106F50007273696F6E206669726D77617265202049
:106F60000020204D454E552020504152414D455462
:106F7000524553202000202020456E7472657220F7
:106F800064616E73206C652020200020202020206A
:106F90006261636B6C696768742020202020200088
:106FA00020202020205265676C6572206C652020AF
:106FB00020202020002064652020666F6E637469A5
:106FC0006F6E6E656D656E742000202020526567BF
:106FD0006C6572206C65206D6F6465202020002038
:106FE0002020205425732020616D6269616E7465D4
:106FF000202020200020202020542573206465704C
:107000006172742050432020202000205265676C5C
:107010006572206C6120636F6E7369676E65200016
:107020003C2D2D202020202020202020202020202A
:10703000202D2D3E002020202020205175697474C1
:107040006572203F202020202000202020202020AA
:1070500020202020202020202020202D2D3E002513
:1070600073002D2D2D2D2D2020204D454E552020F7
:10707000202D2D2D2D2D0053555243484155464668
:1070800045205425732042414C4C4F4E0020504F18
:107090004D50452041204348414C455552204853CE
:1070A000200054454D504552415455524520504CB6
:1070B000414E4348455200534F4E444520454155AB
:1070C0002042414C4C4F4E2020485300534F4E44D9
:1070D000452045585445524945555245202048536E
:1070E0000020534F4E4445204445504152542050B7
:1070F000432048532000202045525245555220201D
:107100004445544543544545202000207261667231
:1071100061696368697373656D656E742E2E2E00E8
:10712000202020206368617566666167652E2E2EBB
:107130002020202000202050617373616765206546
:107140006E206D6F6465202020002D2D2D2D2D2D9E
:107150002D2D2D2D2D2D2D2D2D2D2D2D2D2D004178
:1071600070706F696E742020202020203A20204FFC
:10717000464620004170706F696E742020202020E8
:10718000203A20204F4E20200047726F75706520F6
:107190004578742E20203A20204F46462000477222
:1071A0006F757065204578742E20203A20204F4E50
:1071B00020200047726F757065204578742E203A44
:1071C0002045525245555200542573204561752083
:1071D00042616C6C6F6E3A257325730054257320E1
:1071E0004561752042616C6C6F6E3A2053484F5276
:1071F0005400542573204561752042616C6C6F6E9C
:107200003A204F50454E20005365636F75727320CE
:1072100020737572206170706F696E74002D2D2D52
:107220002D2D204574617420504143202D2D2D2D8E
:107230002D0043697263756C617465757220203A24
:1072400020204F4646200043697263756C61746567
:10725000757220203A20204F4E20200054257320A4
:10726000204465706172742050433A257325730081
:1072700054257320204465706172742050433A2075
:1072800053484F5254005425732020446570617256
:10729000742050433A204F50454E2000436F6E7388
:1072A0002E204465702E2050433A2573257300200C
:1072B00020202020454E2050415553452E2E2E2073
:1072C0002020200056616E6E65203320766F696540
:1072D00073206665726D6565002D2D20457461749F
:1072E0002020506C616E63686572202D2D0054253E
:1072F0007320457874657269657572653A257325E2
:1073000073005425732045787465726965757265DC
:107310003A2053484F5254005425732045787465E1
:107320007269657572653A204F50454E20005425AC
:107330007320416D6269616E746520203A25732562
:10734000730054257320416D6269616E746520205D
:107350003A2053484F52540054257320416D6269BE
:10736000616E746520203A204F50454E2000436FD7
:107370006E7369676E6520416D622E3A25732573C1
:10738000002D2D2D2D2D20204152524554202020FE
:107390002D2D2D2D2D002D2D2D2D204D6F64652093
:1073A00046726F6964202D2D2D2D002D2D204D6FDF
:1073B000646520436861756666616765202D2D00F0
:1073C000D88801D0D8984AE8D9CFE6FFDACFE6FFCF
:1073D000E1CFD9FFE2CFDAFF94E9D8B8037E086A9B
:1073E000E2EC3AF0FAEC3AF008B6C6EF3AF008A24E
:1073F0000AD008AA03D008BEC6EF3AF008A4D2EF1C
:107400003AF0CFEF3AF008AA05D008ACD2EF3AF044
:10741000CFEF3AF008A00AD008A808D008BE04D0E0
:1074200008A402D0DBEF3AF0DFEF3AF0096A0E6A07
:107430000350075C106E10E384EB0AF085EB0BF051
:1074400086EB0CF087EB0FF080EB04F081EB05F09E
:1074500082EB06F0083A09D080EB0AF081EB0BF0E2
:1074600082EB0CF083EB0FF0106C089E08BC088ECA
:107470008FEB0DF008B0B1EF3AF01A0E1060B1EFDB
:107480003AF00D6A076A08A408D0046C051E061EAF
:10749000071EE86A05220622072208AC08D00A6CFB
:1074A0000B1E0C1E0D1EE86A0B220C220D22116A07
:1074B000105207E007340632053204321132102E22
:1074C000F9D704500A2605500B2206500C2207500B
:1074D0000D2291EB09F0089E0DAE0BD0096C0A1E2F
:1074E0000B1E0C1E0D1EE86A0A220B220C220D2216
:1074F000088E0DA006D0D8800C320B320A32093229
:107500000F2A8FEB0DF085EF3AF00C500B100A109C
:10751000091055E00EBE4DD00CBE0CD00D500E1013
:1075200048E0D89009360A360B360C360D06D8A03E
:107530000E06F2D70E5031E10D282FE009AE11D022
:107540007F0E091402E10AA00CD00A2AE86A0B2275
:107550000C2207E3D8800C320B320A320D2A0D2898
:107560001CE00D5026E08AEB00F08BEB01F00C34B0
:10757000026E0D30036E0232039E08BE038EE5528A
:10758000E5CFDAFFE7CFD9FF4EE912007F0E036E99
:10759000FF0E026E016E006EF2D77F0E08BEFF0E68
:1075A000036E02D07F0E036E800E026E016A006AC7
:1075B000E6D708AE04D0800E036E026AF7D7036ADE
:1075C000026AF4D70636073602E30884087E06E12D
:1075D0000880076A066A056A046A1200072803E041
:1075E000D88006321200D890063202E108821200DA
:1075F000088612000236033602E3088C087E06E194
:107600000888036A026A016A006A1200032803E01C
:10761000D88002321200D8900232EAE1088A1200C1
:10762000D89801D0D88851E8D9CFE6FFDACFE6FF65
:10763000E1CFD9FFE2CFDAFF94E9089E04E700AE7C
:1076400002D0006C088E80EB0CF00B6A0A6A096AA3
:10765000860E0D6E0E6A85EF3AF0D89801D0D88864
:1076600050E8D9CFE6FFDACFE6FFE1CFD9FFE2CF8E
:10767000DAFF94E9089E07E701AE05D0006C011E11
:10768000E86A0122088E81EB0CF080EB0BF00A6AAD
:10769000096A8E0E0D6E0E6A85EF3AF045E8D9CF75
:1076A000E6FFDACFE6FFE1CFD9FFE2CFDAFF8BE9E1
:1076B000086AFAEC3AF008B662EF3BF008AA0ED07E
:1076C00008BC05D07F0E016EFF0E006E23D0800E29
:1076D000016E006A1FD0016A006A1CD008B8FBD78F
:1076E0008F0E0360EDD77E0E0364F5D78E0E035C1C
:1076F00005E0D89002320132032AF8D708AC06D050
:10770000016C021EE86A022202AEE5D781EB00F0AE
:1077100082EB01F0E552E5CFDAFFE7CFD9FF47E989
:10772000120043E8D9CFE6FFDACFE6FFE1CFD9FF79
:10773000E2CFDAFF89E9066A1200F3DF068001D0A2
:10774000F0DF01AEAAEF3BF0006C011EE86A0122F7
:1077500006B0067E03AEB2EF3BF0026C031EE86A91
:107760000322067E62EC3DF003BED4EF3BF006AE92
:1077700008D0026C031EE86A0322046C051EE86A46
:10778000052206B006D084EB00F085EB01F006A0E0
:1077900004D082EB00F083EB01F0E552E5CFDAFF95
:1077A000E7CFD9FF45E9000C06BEB9EF3BF0E9DFB2
:1077B000FF0C4AE8D9CFE6FFDACFE6FFE1CFD9FFE9
:1077C000E2CFDAFF94E9086AE2EC3AF0FAEC3AF038
:1077D00008B6C6EF3AF008A205D008BAC6EF3AF0EC
:1077E000CDEF3AF008BAD9EF3AF008A005D008B8C2
:1077F000C6EF3AF0D9EF3AF008B8CDEF3AF00E6A9A
:107800007F0E07240D6EE86A0E2203500D5EE86AB3
:107810000E5A1A0E0F6E076A096A0A6A0B6A0C6A18
:107820000050045E0150055A0250065A000E075AD5
:1078300009E7005004260150052202500622000EDE
:10784000072201D0098AD890043605360636073655
:10785000D89009360A360B360C360F2EE1D7065073
:1078600005100410D8A4098A85EF3AF03FEC3CF0EB
:10787000E8B6000CE8B0000CE8A4000C010C47E8E6
:10788000D9CFE6FFDACFE6FFE1CFD9FFE2CFDAFFCB
:1078900091E9086AE2EC3AF0FAEC3AF008B64ED018
:1078A00008AE08D008A004D008A802D0088046D0AE
:1078B000089044D00350075C0BE10250065C08E1DD
:1078C0000150055C05E10050045C02E1088036D0FF
:1078D000D8A002D0088E10D007500318071A031A38
:1078E00006500218061A021A05500118051A011A44
:1078F00004500018041A001A0350075C10E0FF0F30
:1079000009E0089008B403D008AE088417D008AE88
:10791000089414D0032AD890023201320032005069
:10792000045E0150055A0250065A06BEEAD7D890A6
:10793000043605360636072EF8D7C8D70850E55264
:10794000E5CFDAFFE7CFD9FF4FE9120044E8D9CFFE
:10795000E6FFDACFE6FFE1CFD9FFE2CFDAFF8AE92F
:1079600080EB04F081EB05F082EB06F0025004029C
:10797000F450016EF350006E0350076E0502F45090
:10798000036EF350026E07500402F3500126F450C8
:107990000222E86A032206500502F3500126F45041
:1079A0000222E86A0322E552E5CFDAFFE7CFD9FFEA
:1079B00046E9000C4AE8D9CFE6FFDACFE6FFE1CF8F
:1079C000D9FFE2CFDAFF94E9086AE2EC3AF0FAEC88
:1079D0003AF008B6C6EF3AF008A205D008B8C6EFEC
:1079E0003AF0CDEF3AF008AA05D008B0C6EF3AF069
:1079F000CDEF3AF008B002D008A802D0D9EF3AF0A3
:107A00000E6A035007240D6EE86A0E227E0E0D5E8C
:107A1000E86A0E5A096A0A6A0B6A0C6A0250060280
:107A2000F4500C6EF3500B6E01500602F3500A2610
:107A3000F4500B22000E0C2202500502F3500A26CD
:107A4000F4500B22000E0C2200500602F3500926BF
:107A5000F4500A22000E0B220C2201500502F350B2
:107A60000926F4500A22000E0B220C2202500402B6
:107A7000F3500926F4500A22000E0B220C2200506B
:107A80000502F4500926000E0A220B220C22015096
:107A90000402F4500926000E0A220B220C2285EF64
:107AA0003AF043E8D9CFE6FFDACFE6FFE1CFD9FFDE
:107AB000E2CFDAFF89E9066A1200F3DF068003D01D
:107AC000F0DF01D00682056A046A100EE76ED890D6
:107AD00002360336043605360050045C0150055862
:107AE00005E30050045E0150055A022AE72EF0D744
:107AF00006B2120006B006D084EB00F085EB01F070
:107B000006A004D082EB00F083EB01F0E552E5CF54
:107B1000DAFFE7CFD9FF45E9120045E8D9CFE6FF04
:107B2000DACFE6FFE1CFD9FFE2CFDAFF8FE90C6AC7
:107B30001200F3DF0C8003D0F0DF01D00C820B6A5F
:107B40000A6A096A086A200EE76ED890043605367C
:107B500006360736083609360A360B360050085CFA
:107B60000150095802500A5803500B5809E30050BD
:107B7000085E0150095A02500A5A03500B5A042A4F
:107B8000E72EE4D70CB212000CB00AD088EB00F05C
:107B900089EB01F08AEB02F08BEB03F00CA008D02C
:107BA00084EB00F085EB01F086EB02F087EB03F04D
:107BB000E552E5CFDAFFE7CFD9FF49E9120044E803
:107BC000D9CFE6FFDACFE6FFE1CFD9FFE2CFDAFF88
:107BD0008EE980EB08F081EB09F082EB0AF083EB91
:107BE0000BF004500802F350006EF450016E045084
:107BF0000902F3500126000EF420026E04500A021E
:107C0000F3500226000EF420036E04500B02F350D2
:107C1000032605500802F3500126F4500222000EFC
:107C2000032205500902F3500226F45003220550A6
:107C30000A02F350032606500802F3500226F450BD
:107C4000032206500902F350032607500802F3509E
:107C50000326E552E5CFDAFFE7CFD9FF48E9000C6C
:107C6000D9CFE6FFE1CFD9FF81E942E8E668050E0A
:107C7000E66EE66A1FEC4AF043E970EC4CF006C091
:107C8000E6FF000EE66EE66A1FEC4AF043E970EC90
:107C90004CF007C0E6FF010EE66EE66A1FEC4AF004
:107CA00043E970EC4CF0080E016E000E026E01EB21
:107CB000E9FF02EBEAFFEFCFE6FF020EE66EE66AAF
:107CC0001FEC4AF043E970EC4CF00128E96E000E1D
:107CD0000220EA6EEFCFE6FF030EE66EE66A1FECC7
:107CE0004AF043E970EC4CF048C0E6FF040EE66E43
:107CF000E66A1FEC4AF043E970EC4CF0550EE66E74
:107D0000050EE66EE66A1FEC4AF043E943E9E7CF69
:107D1000D9FF1200D9CFE6FFE1CFD9FF81E942E8D0
:107D2000E6681B0EE66EE66A1FEC4AF043E970EC6B
:107D30004CF00A0E016E000E026E01EBE9FF02EB41
:107D4000EAFFEFCFE6FF060EE66EE66A1FEC4AF0AA
:107D500043E970EC4CF00128E96E000E0220EA6E57
:107D6000EFCFE6FF070EE66EE66A1FEC4AF043E946
:107D700070EC4CF00C0E016E000E026E01EBE9FF90
:107D800002EBEAFFEFCFE6FF080EE66EE66A1FECB5
:107D90004AF043E970EC4CF00128E96E000E022035
:107DA000EA6EEFCFE6FF090EE66EE66A1FEC4AF0D8
:107DB00043E970EC4CF00E0E016E000E026E01EB0A
:107DC000E9FF02EBEAFFEFCFE6FF0A0EE66EE66A96
:107DD0001FEC4AF043E970EC4CF00128E96E000E0C
:107DE0000220EA6EEFCFE6FF0B0EE66EE66A1FECAE
:107DF0004AF043E970EC4CF010C0E6FF0C0EE66E62
:107E0000E66A1FEC4AF043E970EC4CF011C0E6FF63
:107E10000D0EE66EE66A1FEC4AF043E970EC4CF09A
:107E200012C0E6FF0E0EE66EE66A1FEC4AF043E96A
:107E300070EC4CF013C0E6FF0F0EE66EE66A1FEC26
:107E40004AF043E970EC4CF014C0E6FF100EE66E09
:107E5000E66A1FEC4AF043E970EC4CF015C0E6FF0F
:107E6000110EE66EE66A1FEC4AF043E970EC4CF046
:107E700016C0E6FF120EE66EE66A1FEC4AF043E912
:107E800070EC4CF017C0E6FF130EE66EE66A1FECCE
:107E90004AF043E970EC4CF01EC0E6FF140EE66EAB
:107EA000E66A1FEC4AF043E970EC4CF0180E016EE4
:107EB000000E026E01EBE9FF02EBEAFFEFCFE6FFF7
:107EC000150EE66EE66A1FEC4AF043E970EC4CF0E2
:107ED0000128E96E000E0220EA6EEFCFE6FF160ED3
:107EE000E66EE66A1FEC4AF043E970EC4CF01A0EBD
:107EF000016E000E026E01EBE9FF02EBEAFFEFCF2D
:107F0000E6FF170EE66EE66A1FEC4AF043E970ECF6
:107F10004CF00128E96E000E0220EA6EEFCFE6FF7A
:107F2000180EE66EE66A1FEC4AF043E970EC4CF07E
:107F30001C0E016E000E026E01EBE9FF02EBEAFF80
:107F4000EFCFE6FF190EE66EE66A1FEC4AF043E952
:107F500070EC4CF00128E96E000E0220EA6EEFCFC3
:107F6000E6FF1A0EE66EE66A1FEC4AF043E970EC93
:107F70004CF0550EE66E1B0EE66EE66A1FEC4AF0FC
:107F800043E9E668080EE66E030EE66E1FEC4AF063
:107F900043E970EC4CF0230E016E000E026E01EB13
:107FA000E9FF02EBEAFFEFCFE6FFE66A030EE66EBB
:107FB0001FEC4AF043E970EC4CF00128E96E000E2A
:107FC0000220EA6EEFCFE6FF010EE66E030EE66ECC
:107FD0001FEC4AF043E970EC4CF0290E016E000EE4
:107FE000026E01EBE9FF02EBEAFFEFCFE6FF020EC4
:107FF000E66E030EE66E1FEC4AF043E970EC4CF0BF
:108000000128E96E000E0220EA6EEFCFE6FF030EB4
:10801000E66E030EE66E1FEC4AF043E970EC4CF09E
:108020002F0E016E000E026E01EBE9FF02EBEAFF7C
:10803000EFCFE6FF040EE66E030EE66E1FEC4AF08D
:1080400043E970EC4CF00128E96E000E0220EA6E64
:10805000EFCFE6FF050EE66E030EE66E1FEC4AF06C
:1080600043E970EC4CF0350E016E000E026E01EB30
:10807000E9FF02EBEAFFEFCFE6FF060EE66E030E26
:10808000E66E1FEC4AF043E970EC4CF00128E96E13
:10809000000E0220EA6EEFCFE6FF070EE66E030E3B
:1080A000E66E1FEC4AF043E970EC4CF0550EE66EBC
:1080B000080EE66E030EE66E1FEC4AF043E943E954
:1080C000E7CFD9FF1200D9CFE6FFE1CFD9FF81E991
:1080D00042E8050EE66EE66AE8EC4AF042E9550829
:1080E00039E1000EE66EE66AE8EC4AF042E900018A
:1080F000066F010EE66EE66AE8EC4AF042E900011E
:10810000076F080E016E000E026E020EE66EE66A42
:10811000E8EC4AF042E9E66E01EBE9FF02EBEAFF28
:10812000E552E750EF6E030EE66EE66AE8EC4AF0C1
:1081300042E9E66E0128E96E000E0220EA6EE55281
:10814000E750EF6E040EE66EE66AE8EC4AF042E9AC
:108150000001486F1B0EE66EE66AE8EC4AF042E961
:10816000550801E00ED10A0E016E000E026E060ED9
:10817000E66EE66AE8EC4AF042E9E66E01EBE9FFFA
:1081800002EBEAFFE552E750EF6E070EE66EE66A95
:10819000E8EC4AF042E9E66E0128E96E000E0220A2
:1081A000EA6EE552E750EF6E0C0E016E000E026EA5
:1081B000080EE66EE66AE8EC4AF042E9E66E01EB8C
:1081C000E9FF02EBEAFFE552E750EF6E090EE66EBB
:1081D000E66AE8EC4AF042E9E66E0128E96E000E34
:1081E0000220EA6EE552E750EF6E0E0E016E000EB1
:1081F000026E0A0EE66EE66AE8EC4AF042E9E66EC6
:1082000001EBE9FF02EBEAFFE552E750EF6E0B0EE0
:10821000E66EE66AE8EC4AF042E9E66E0128E96EAD
:10822000000E0220EA6EE552E750EF6E0C0EE66E8D
:10823000E66AE8EC4AF042E90001106F0D0EE66EC6
:10824000E66AE8EC4AF042E90001116F0E0EE66EB4
:10825000E66AE8EC4AF042E90001126F0F0EE66EA2
:10826000E66AE8EC4AF042E90001136F100EE66E90
:10827000E66AE8EC4AF042E90001146F110EE66E7E
:10828000E66AE8EC4AF042E90001156F120EE66E6C
:10829000E66AE8EC4AF042E90001166F130EE66E5A
:1082A000E66AE8EC4AF042E90001176F140EE66E48
:1082B000E66AE8EC4AF042E900011E6F180E016E12
:1082C000000E026E150EE66EE66AE8EC4AF042E930
:1082D000E66E01EBE9FF02EBEAFFE552E750EF6ED5
:1082E000160EE66EE66AE8EC4AF042E9E66E012810
:1082F000E96E000E0220EA6EE552E750EF6E1A0EAC
:10830000016E000E026E170EE66EE66AE8EC4AF0A9
:1083100042E9E66E01EBE9FF02EBEAFFE552E750C6
:10832000EF6E180EE66EE66AE8EC4AF042E9E66E99
:108330000128E96E000E0220EA6EE552E750EF6E6A
:108340001C0E016E000E026E190EE66EE66AE8EC77
:108350004AF042E9E66E01EBE9FF02EBEAFFE55283
:10836000E750EF6E1A0EE66EE66AE8EC4AF042E974
:10837000E66E0128E96E000E0220EA6EE552E75033
:10838000EF6E080EE66E030EE66EE8EC4AF042E988
:10839000550801E08BD0230E016E000E026EE66AD6
:1083A000030EE66EE8EC4AF042E9E66E01EBE9FF07
:1083B00002EBEAFFE552E750EF6E010EE66E030EA8
:1083C000E66EE8EC4AF042E9E66E0128E96E000E3E
:1083D0000220EA6EE552E750EF6E290E016E000EA4
:1083E000026E020EE66E030EE66EE8EC4AF042E91B
:1083F000E66E01EBE9FF02EBEAFFE552E750EF6EB4
:10840000030EE66E030EE66EE8EC4AF042E9E66E15
:108410000128E96E000E0220EA6EE552E750EF6E89
:108420002F0E016E000E026E040EE66E030EE66E57
:10843000E8EC4AF042E9E66E01EBE9FF02EBEAFF05
:10844000E552E750EF6E050EE66E030EE66EE8ECC1
:108450004AF042E9E66E0128E96E000E0220EA6E5B
:10846000E552E750EF6E350E016E000E026E060EFD
:10847000E66E030EE66EE8EC4AF042E9E66E01EBCA
:10848000E9FF02EBEAFFE552E750EF6E070EE66EFA
:10849000030EE66EE8EC4AF042E9E66E0128E96E6A
:1084A000000E0220EA6EE552E750EF6E43E9E7CF97
:0484B000D9FF1200DE
:0C84B40090DB86E90150010600090CE095
:1084C00002EBE6FF03EBE6FF00EBE6FF69DBF4E11E
:1084D000DC1DF2E1010E01D0000E41E9E5CFDAFF2B
:1084E000E7CFD9FF120077DB89E97BE80A6A0B6ADC
:1084F00002EBF6FF03EBF7FF04EBF8FF0800F55083
:10850000096E095001E12DD3250E095C01E01BD352
:108510000C6A0D6A0E6A0F6A106A2DDB2D0E095C5B
:108520000CE02B0E095C09E0200E095C06E0230E2E
:10853000095C03E0300E095C15E10950300A10E0D7
:10854000130A0CE0030A08E00B0A04E0060AE5E15E
:108550000C80E3D70C82E1D70C84DFD70C86DDD703
:108560000C88DBD72A0E095C13E1A5DB0DE30C8038
:108570001CEBDBF01DEBDCF00001DB6DDC1F000E03
:10858000DC23DB510D6E02D09CEB0DF0F4DA07D04A
:10859000126A3FDB02E06BDBFCD792EB0DF00CB014
:1085A0000C982E0E095C15E1E6DA2A0E095C08E14A
:1085B00082DB04E29CEB0EF0010E0F6EDCDA09D0D8
:1085C000126A27DB02E053DBFCD792EB0EF0010EC0
:1085D0000F6E680E095C07E1CEDA680E095C1DE1DA
:1085E000030E106E19D0740E095C16E07A0E095C49
:1085F00013E0480E095C06E0540E095C03E05A0ED5
:10860000095C02E1020E07D06C0E095C03E06A0E01
:10861000095C03E1010E106EAEDA09506E0A01E149
:108620006ED21E0A01E128D1200A01E125D13F0ABC
:1086300001E1FDD01A0A01E1FAD00D0A01E1F7D0FB
:10864000200A01E1F4D03A0A01E1F1D0200A01E167
:10865000EED0260A01E1EAD00D0A01E1E7D01A0ABC
:1086600001E19ED0200A3BE0300A1AE0460A0EE003
:10867000250A01E072D2D950020FE96E000EDA200D
:10868000EA6E010EEE5E000EEE5AEE5A0FDB250E7C
:10869000E66E86DA03E1DC1D01E159D20A2A5BD2DB
:1086A000116A0D50010803E20D04116EF5DA115044
:1086B00007E0010E0C1404E16DDA01E048D2116A02
:1086C000D3DAEF50096ECBDA03E1DC1D01E13FD2D2
:1086D0000A2A000E0B225EDA01E13FD238D2020EE6
:1086E000105C08E1030E4EDAEE50176EEE50186E75
:1086F000EF5007D0E7DADD6BDB51176EDC51186EF7
:10870000DD51196E17EBE6FF18EBE6FF19EBE6FFFC
:10871000C7EC49F043E9E2C0DBF0E3C0DCF0E4C0C1
:10872000DDF00001DB511C6EDC511D6E0F5006E0C8
:108730001C500E5C03E20E501C6E1D6A1C500D5C3A
:1087400002E29CEB0DF050DA05E00D500E5C02E207
:108750008EEB0DF00CB004D01DDA01E0F8D1116AF7
:10876000126A17EBF6FF18EBF7FF19EBF8FF08009A
:10877000F550096E095010E00D50125C0DE26FDAF1
:1087800003E1DC1D01E1E3D10A2A000E0B22122ACB
:10879000D950170F55DAEBD7FDD901E1DED1D7D18A
:1087A00063DAEE501A6EED501B6E1AEBE6FF1BEB10
:1087B000E6FFB9EC49F042E9F3501C6EF4501D6E2F
:1087C0000F5006E01C500E5C03E20E501C6E1D6A3A
:1087D0001C500D5C02E29CEB0DF006DA05E00D503A
:1087E0000E5C02E28EEB0DF00CB004D0D3D901E0A8
:1087F000AED1116A126A1AEBE9FF1BEBEAFFEF50E8
:10880000096E09500FE00D50125C0CE228DA03E10A
:10881000DC1D01E19CD10A2A000E0B22122A1A2A21
:108820001B22E9D7B7D901E198D191D10C8E100460
:108830000AE1040EA7D9EE50136EEE50146EEE50FE
:10884000156EEF5032D0030E105C16E10CAE0CD05A
:108850000BDAEFCFDBF00001DC6BDD6BDE6BDBAF47
:1088600023D0DC69DD691FD0FFD9EFCFDBF0000139
:10887000DB51136E146A20D0020E105C0CE10CAEBA
:1088800006D0030E7FD9B6D9DDAF0ED00CD0030EC3
:1088900079D9B0D909D00CAE0AD014DADD6BDE6B11
:1088A000DCAF02D0DD69DE69BCD9166E07D00ADA0A
:1088B000DB51136EDC51146E156A166A0F5002E11B
:1088C000010E0E6E1E6A1F6AD950400FE66E000E32
:1088D000DA20E66EE552E550436EE750426E416A9B
:1088E000116A0A0E106E0950780A12E0200A10E090
:1088F000280A0CE0200A0AE03F0A06E00D0A02E01E
:10890000200A08E1020E05D0080E03D0080E092641
:10891000100E106E0CBE02D00C920C94800E0C1433
:1089200017E0163415E3E668E668E668E66842D9BB
:10893000DFEC3DF0E552E5CFDEF0E5CFDDF0E5CF51
:10894000DCF0E7CFDBF000016CD9166E2D0E07D0FE
:108950000CA202D02B0E03D00CA404D0200E206E4B
:108960001E2A01D0206A0E5005E113501410151074
:10897000161061E00001BC0EDB6F980EDC6F000E7C
:10898000DD6F83D99CEC3DF0E552E5CFE1F0E5CF1A
:10899000E0F0E5CFDFF0E7CFDEF00001DB51DE25D0
:1089A000F36EDC51DF21F46EDD51E021F86EF4CF7F
:1089B000F7FFF3CFF6FF0800F550126E580E095C72
:1089C00005E1610E125C02E3200E125E5ED999ECA5
:1089D0003DF0E552E550166EE550156EE550146E0B
:1089E000E750136E42EBE9FF43EBEAFF4206000E4D
:1089F000435A12EBEFFF1E2A1350141015101610D5
:108A0000B9E10CA619D06F0E095C06E10E501E5C90
:108A100013E31E280E6E10D0780E095C09E0580E84
:108A2000095C06E0620E095C03E0420E095C04E1A9
:108A3000020E1F6E01D01E6A100E0C1407E00D50BE
:108A40000E5C04E20F5002E18DEB0EF00E501E5C46
:108A500003E21E500E5E01D00E6A0E501E241F242B
:108A6000D8800D5407E20E500D5CD8801E54D8807B
:108A70001F54116E010E0C1406E1115004E08AD847
:108A800066E10AD9116A205007E010D920EBE6FF11
:108A900087D802E1DC1D5BE01F500BE007D9300EE8
:108AA000E66E7ED802E1DC1D52E0D9D802E1DC1D81
:108AB0004EE00E501F5C02E21F500E5E300EE66E5E
:108AC0000EEBE6FFDCD843E1422A000E432242EBE4
:108AD000E9FF43EBEAFFEF50126E125008E0E6D8D0
:108AE00012EBE6FF5DD8F0E1DC1DEEE130D052D8AC
:108AF0002EE10E501E2411241F240A262CD01050C3
:108B0000030A1CE0010A14E0030A07E0ADD8C9D843
:108B10000AEBEEFF0BEBEDFF20D08BD8DE6BDCAF6A
:108B200002D0DD69DE69A0D84ED8DEC0EEFF15D0D8
:108B300080D8DCBFDD6998D846D80FD095D8B1D899
:108B40000AEBEFFF0AD08BD805E1DC1D03E1F368E7
:108B5000F4680BD00A2A000E0B22D950020F70D8ED
:108B6000CDD40AEBF3FF0BEBF4FF7CE9E5CFDAFFA2
:108B7000E7CFD9FF1200D950020F62D80800F55094
:108B8000096E1200005E000E015A00EBE9FF01EBD6
:108B9000EAFF1200200EE66E11EBE6FF3FEF46F013
:108BA000ECEC49F043E9F3CFDBF0F4CFDCF000016B
:108BB000F31C120013EBE6FF14EBE6FF15EBE6FFE8
:108BC00016EBE6FF12006DD8DBC0EEFFDCC0EEFF57
:108BD000DDC0EEFF1200D9CFE6FFDACFE6FFE1CF2E
:108BE000D9FFE2CFDAFF12001C500D5C116E54D891
:108BF0000F501200EECFDBF0EECFDCF0EFCFDDF068
:108C00000001DE6B1200EECFDBF0EFCFDCF00001F5
:108C100012000950E66EE66AFAEC4BF042E9F350B6
:108C20001200DB51136EDC51146EDD51156EDE51F6
:108C300012000AEBDBF00BEBDCF00001DD6B120045
:108C4000E96E000EDA20EA6EEF2AEECFF6FF000E94
:108C5000EF22EECFF7FFEF22EECFF8FF120026D87B
:108C600009EBE6FFD0EF45F0020EC2EF45F00A0E29
:108C70001202F3500924D00F126EBBEF45F016D844
:108C80005AEC42F044E90009120010EBE6FFE66AF4
:108C9000E66AE66ADAEF45F011500A26000E0B226A
:108CA0001200EE50EFCFEAFFE96E120005EBE6FF8F
:108CB00006EBE6FF1200D8DFEE501C6EED501D6E85
:0A8CC0001D341200D1DF03EF46F06F
:068CCA000CD911D924D9D8
:108CD00057D94AD969D912000001006B0001010E71
:108CE000016F000102690001036B0001046B056B59
:108CF0000001476B0001020E486F0001496B000143
:108D0000066B0001020E076FC80E0001086F096BA9
:108D10000001FC0E0A6F0B6900010E0E0C6F010EB4
:108D20000D6F0001F40E0E6F010E0F6F00011E0E8D
:108D3000106F0001CE0E116F00010F0E126F0001B7
:108D4000140E136F0001146B0001050E156F000166
:108D5000010E166F0001176B640E0001186F196B7E
:108D6000780E00011A6F1B6B00012C0E1C6F010E98
:108D70001D6F0001640E1E6F0001010E376F0001B0
:108D8000010E386F0001010E396FC80E00013A6FF5
:108D90003B6B00013C6B00013D6B00013E6B000131
:108DA0003F6B406B0001416B426B0001436B446BB6
:108DB000640E0001456F466B0001010E4A6F000111
:108DC000020E4B6F00014C6B0001030E4D6F120041
:108DD000D9CFE6FFE1CFD9FF81E946E8830EE66E01
:108DE000D0EC4BF041E973EC4CF067EC4CF000092F
:108DF00001E0FBD747EC4CF0F3CF1FF0F4CF20F0AD
:108E00001FC0E6FF20C0E6FF86EC31F042E9F3CF59
:108E100021F0F4CF22F00001236B246B870EE66E65
:108E2000D0EC4BF041E973EC4CF067EC4CF00009EE
:108E300001E0FBD747EC4CF0F3CF25F0F4CF26F060
:108E400025C0E6FF26C0E6FF86EC31F042E9F3CF0D
:108E500027F0F4CF28F00001296B2A6B8B0EE66E09
:108E6000D0EC4BF041E973EC4CF067EC4CF00009AE
:108E700001E0FBD747EC4CF0F3CF2BF0F4CF2CF014
:108E80002BC0E6FF2CC0E6FF86EC31F042E9F3CFC1
:108E90002DF0F4CF2EF000012F6B306B930EE66EA9
:108EA000D0EC4BF041E973EC4CF067EC4CF000096E
:108EB00001E0FBD747EC4CF0F3CF31F0F4CF32F0C8
:108EC00031C0E6FF32C0E6FF86EC31F042E9F3CF75
:108ED00033F0F4CF34F00001356B366B47E9E7CF60
:108EE000D9FF12008F0ED3147009D36ED3821200F3
:108EF000806A3F0E926E816A9380938293849396E8
:108F00009398939A826A400E946E836A9568846AF5
:108F10009680969296841200D9CFE6FFE1CFD9FFD2
:108F200081E943E8016A026A036ADF0E016E030EFB
:108F3000026E100E036E03EBE6FF02EBE6FF01EBA1
:108F4000E6FF51EC4AF043E90F015D9B0F015D9D87
:108F50000F015D9F0F015C910F015C930F015C9508
:108F600044E9E7CFD9FF1200380EE66E68EC48F00E
:108F700041E9DAEC1CF0E66AC7EC1CF041E91200AA
:108F800099900B0EBB6E500EBC6EC30EBD6E7F0E65
:108F9000E66E1B0EE66E7DEC4AF042E9D40EE66EFC
:108FA00024EC4BF041E91200D08EA382A582F28E10
:028FB0001200AD
:0E8FB200DACFE4FFE2CFDAFFF3CFE4FFF4CF33
:108FC000E4FFE652D9CFE6FFE1CFD9FF81E942E8DD
:108FD000A4A248D000014951000802E2000149075B
:108FE00000014A2B00014B2B00014C2B00014D2BA3
:108FF00000015F2B050E00015F5D07E300015F6B61
:1090000000010329010B0001036F00013C0507E18A
:1090100000013E0504E100013F2B000E4023020E3B
:1090200000013D5D0EE10001D890445104E6A40E1C
:10903000435D060E445905E20001432B000E442314
:1090400010D0030E00013D5D0CE10001443504E346
:1090500043515C08F90E445504E200014307000E39
:10906000445BA492F2A429D0030E8114016E000186
:109070005E51015C1CE00150040DF35000015E25BF
:10908000026E01EB5EF00250010A0AE00F0A08E0EE
:109090000C0A03E00F0A01E006D00001470704D0E4
:1090A0000001472B01D000D00001640E496F81B44C
:1090B00003D00001640E496FF29443E9E7CFD9FF72
:1090C000E552E5CFF4FFE5CFF3FFE5CFDAFF11007E
:1090D000D9CFE6FFE1CFD9FF82E9836A956A9398F9
:1090E000939A93968A988A9A8A965CEC1DF0300E31
:1090F000E66E71EC4BF041E9050EE66E09EC4BF0C3
:1091000041E9300EE66E71EC4BF041E9010EE66E7E
:1091100009EC4BF041E9320EE66E71EC4BF041E99F
:10912000E7EC4BF0000901E0FBD7E7EC4BF000095E
:1091300001E0FBD700EBE6FF71EC4BF041E9E7EC17
:109140004BF0000901E0FBD7080EE66E71EC4BF026
:1091500041E9E7EC4BF0000901E0FBD70C0EE66EAD
:1091600071EC4BF041E9E7EC4BF0000901E0FBD773
:10917000010EE66E71EC4BF041E9E7EC4BF00009B3
:1091800001E0FBD7060EE66E71EC4BF041E9E7EC2F
:109190004BF0000901E0FBD7800EE66E3FEC4BF090
:0C91A00041E900D041E9E7CFD9FF1200FF
:0491AC001A0EFD0D8D
:1091B000DF0DC00D9F0D7E0D5B0D370D110DEB0CFE
:1091C000C30C9A0C700C450C180CEB0BBD0B8D0BE3
:1091D0005D0B2C0BFA0AC70A930A5F0A2A0AF509E3
:1091E000BF09890953091D09E608B0087908430831
:1091F0000D08D707A1076C0738070407D1069E069C
:109200006C063B060B06DB05AD057F055205270501
:10921000FC04D204AA0482045B0436041104EE03A5
:10922000CB03AA0389036A034B032D031103F50241
:10923000DA02C002A7028F02780261024B023602F4
:1092400022020E02FC01E901D801C701B701A70102
:10925000980189017B016E016101550149013D01C0
:029260003201D9
:0E9262000E0EF66E000EF76E000EF86E000196
:109270000900F550596F0900F5505A6F03E159671D
:1092800001D03DD00900F550546F0900F550556FDD
:109290000900F550566F09000900F550E96E090004
:1092A000F550EA6E090009000900F550576F0900F2
:1092B000F550586F09000900F6CF5BF0F7CF5CF06E
:1092C000F8CF5DF054C0F6FF55C0F7FF56C0F8FF69
:1092D0000001575302E1585307E00900F550EE6EC4
:1092E0005707F8E25807F9D75BC0F6FF5CC0F7FFF5
:1092F0005DC0F8FF00015907000E5A5BBFD712008E
:10930000D9CFE6FFDACFE6FFE1CFD9FFE2CFDAFF30
:1093100087E944E8D9CFE6FFDACFE6FFE552E5502A
:109320000A6EE750096E09EBE6FF0AEBE6FF00EB79
:10933000E6FF01EBE6FF02EBE6FFD950030FE66E16
:10934000000EDA20E66E73EC42F047E9F350076E48
:10935000F450086E03EBE9FF04EBEAFFEF6A07EB5A
:10936000F3FF08EBF4FF45E9E5CFDAFFE7CFD9FFDC
:029370001200E9
:0E937200FE0EE3CFE9FFFF0EE3CFEAFFF36A42
:10938000F46AEE5203E0F34AF42AFBD71200FF0E10
:10939000E3CFF8FFE552FF0EE3CFF7FFE552FF0EF4
:1093A000E3CFF6FFE552E66AE66AE66A0900F5529F
:1093B00009E0FD0EE32A05E1FE0EE32A02E1FF0EBD
:1093C000E32AF4D7FD0EE3CFE2F0FE0EE3CFE3F0A5
:0893D000FF0EE3CFE4F01200F0
:0893D800D9CFE6FFDACFE6FF72
:1093E000E1CFD9FFE2CFDAFF85E9013415E200EBE6
:1093F000E9FF01EBEAFFEECFF3FFEDCFF4FFEE2A3A
:10940000000EEF22F3CFE9FFF4CFEAFF02EBEFFF0C
:10941000EF50F36EF46A0DD0FE0E005C05E102EB36
:10942000E6FF2CEC4CF004D002EBE6FF03EC00F07E
:0E94300041E941E9E5CFDAFFE7CFD9FF1200AD
:02943E00D9CF84
:10944000E6FFDACFE6FFE1CFD9FFE2CFDAFF85E929
:1094500041E8056A000102EBDBF0030EDB15756ED7
:10946000FF0E0114746E00EB73FF7F9E7F9C7F8460
:10947000F250800B01E0010E056EF29E550E7E6EDD
:10948000AA0E7E6E7F827FB2FED70550E8B0F28EC4
:10949000E8A0F29E7F9442E9E5CFDAFFE7CFD9FF5B
:0294A0001200B8
:0E94A200D9CFE6FFDACFE6FFE1CFD9FFE2CF68
:1094B000DAFF85E9C26AC16AC06A7C0E0114C26E15
:1094C00000EBC1FF0250040DF350380B0001DC6FBC
:1094D00002380F0B070BDB6F800E0214DB11DC115F
:1094E000C06E01AE03D09E9C9D8CF28CC28041E97F
:0A94F000E5CFDAFFE7CFD9FF120045
:0694FA00D9CFE6FFDACF36
:10950000E6FFE1CFD9FFE2CFDAFF84E9F30E0014E2
:10951000AA6E7F0E0114E824CD6ECF6ACE6A9E90AB
:1095200001AE02D09D8001D09D909E9400A402D0F7
:109530009D8401D09D94AABEAA86CD8041E9E5CF45
:08954000DAFFE7CFD9FF1200AA
:08954800D9CFE6FFE1CFD9FF06
:1095500083E900EBE9FF01EBEAFFEF5012E0E7ECF3
:109560004BF0000901E0FBD700EBE9FF01EBEAFF5C
:10957000EFCFE6FFB9EC4BF041E9002A000E0122E3
:0C958000E8D700D041E9E7CFD9FF120086
:04958C00D9CFE6FF4E
:10959000E1CFD9FF83E900EBE9FF01EBEAFFEF50F0
:1095A00012E0E7EC4BF0000901E0FBD700EBE9FF2C
:1095B00001EBEAFFEFCFE6FFB9EC4BF041E9002AFF
:1095C000000E0122E8D700D041E9E7CFD9FF120011
:1095D000D9CFE6FFDACFE6FFE1CFD9FFE2CFDAFF5E
:1095E00084E9000101EBDBF0DC6B030E0001DB150D
:1095F000756EFF0E0014746E7F9C7F9E7F8000004E
:109600000000735000D041E9E5CFDAFFE7CFD9FF82
:02961000120046
:0E961200FF0EE3500001E76FEE0E02D0F20EE5
:109620000000E76EE72E12EF4BF00C0E0001E66F24
:10963000E76AE72E19EF4BF0E62F18EF4BF0000129
:08964000E72F0FEF4BF01200C1
:08964800D9CFE6FFDACFE6FFFF
:10965000E1CFD9FFE2CFDAFF83E97F0E0014D56EA8
:10966000D76AD66AF29400AE02D0F28A01D0F29A9A
:0E967000D58E41E9E5CFDAFFE7CFD9FF120032
:02967E00D9CF42
:10968000E6FFE1CFD9FF82E9956A800E0010836E74
:109690008A988A9A4EEC1DF08A864EEC1DF08A96C6
:1096A0004EEC1DF0956800D041E9E7CFD9FF1200DC
:1096B000D9CFE6FFE1CFD9FF82E9956A400E0010CD
:1096C000836E8A988A9A4EEC1DF08A864EEC1DF0C5
:1096D0008A964EEC1DF0956800D041E9E7CFD9FF9E
:0296E000120076
:0E96E200D9CFE6FFE1CFD9FF82E9956A00EB10
:1096F00083FF8A988A9A4EEC1DF08A864EEC1DF004
:109700008A964EEC1DF0956800D041E9E7CFD9FF6D
:02971000120045
:0E971200D9CFE6FFE1CFD9FF81E941E88A8A8D
:109720008A884EEC1DF08A864EEC1DF08350016E47
:109730008A968A9A8A98015000D042E9E7CFD9FFE9
:02974000120015
:0E974200D9CFE6FFE1CFD9FF81E941E88A885F
:109750008A9A4EEC1DF08A864EEC1DF08350016E05
:109760008A968A987F0E011400D042E9E7CFD9FF8C
:029770001200E5
:0E977200D9CFE6FFE1CFD9FF82E9956A00EB7F
:1097800083FF8A8A8A984EEC1DF08A864EEC1DF083
:109790008A968A9A956800D041E9E7CFD9FF1200EE
:1097A000D9CFE6FFDACFE6FFE1CFD9FFE2CFDAFF8C
:1097B00083E97C0E00140001DB6F830EC214DB1101
:0E97C000C26E41E9E5CFDAFFE7CFD9FF120014
:0297CE008A8887
:1097D0008A9A4EEC1DF08A864EEC1DF083AE05D0C1
:1097E0008A968A98010E05D004D08A968A98000E2F
:0497F00000D0120093
:0C97F400F36AF46AFF0EE124E96EFF0E38
:10980000E220EA6EED6607D02F0EEF6404D03A0E28
:08981000EF6001D0F32A120001
:08981800FF0EE3500001E76FB1
:10982000480E01D04C0EE76EE72EFED7E76AE72E12
:08983000FED7E72FF7D7120065
:08983800410EF36E00EE00F09A
:109840000E0E01D81200EA6002D0EE6AFCD7F35087
:08985000E9601200EE6AFCD78A
:08985800FF0EE350ACBA04D08E
:10986000AF6AAB8EAC8A949CACA2FED7AD6EF36EA1
:04987000F46A120084
:0C9874001DEE00F02DEE00F0F86A31EC63
:0E98800049F075EC4CF0B4EC28F0FBD7120068
:02988E00C4CF45
:10989000DDF0DDC0DEF00001DD6BC350DD11F36EE5
:0698A000DEC0F4FF12001F
:0A98A600FF0EE350E84E1200000030
:0C98B00000D000D000D0E82EFAD7120043
:0498BC0030313233E2
:0D98C00034353637383961626364656600FF
:0298CE00C25086
:0898D000020B01E0010E120081
:0898D800081408030404030056
:0698E0007FB2FED712006A
:0498E600C282120028
:0298EA0012006A
:0298EC0000007A
:0298EE00010077
:1098F0002020202020202020202020202020202068
:059900002020202000E2
:020000040030CA
:0100000055AA
:0100010008F6
:010002007F7E
:010003007C80
:010005008872
:010006009168
:010008000FE8
:01000900C036
:01000A000FE6
:01000B00E014
:01000C000FE4
:01000D0040B2
:00000001FF
